:020000040000FA
:040800003CEF0CF0CD
:1008100003B275EF05F0F2B493EF05F09EB09BEFD5
:1008200005F09EB2A3EF05F0F2A81AEF04F0F2B2C1
:1008300023EF04F0F2B01FEF04F0EBEF0BF0F296B1
:10084000F290EBEF0BF0CD90F2929EA02DEF04F022
:100850000101533F2DEF04F0542BB2C1B6F1B3C1E7
:10086000B7F1B4C1B8F1B5C1B9F1AEC1B2F1AFC120
:10087000B3F1B0C1B4F1B1C1B5F1AAC1AEF1ABC130
:10088000AFF1ACC1B0F1ADC1B1F1A6C1AAF1A7C140
:10089000ABF1A8C1ACF1A9C1ADF1A2C1A6F1A3C150
:1008A000A7F1A4C1A8F1A5C1A9F19EC1A2F19FC160
:1008B000A3F1A0C1A4F1A1C1A5F19AC19EF19BC170
:1008C0009FF19CC1A0F19DC1A1F1CECF9AF1CFCFF4
:1008D0009BF153C19CF154C19DF1CF6ACE6A0101D5
:1008E000536B546B9E90CD800FBC0F8E0FBA7CEF74
:1008F00004F00F8AEBEF0BF013880F8C0FBEB9EFEB
:1009000004F09AC19EF19BC19FF19CC1A0F19DC1D1
:10091000A1F19EC1A2F19FC1A3F1A0C1A4F1A1C107
:10092000A5F1A2C1A6F1A3C1A7F1A4C1A8F1A5C1D7
:10093000A9F1A6C1AAF1A7C1ABF1A8C1ACF1A9C1A7
:10094000ADF1AAC1AEF1ABC1AFF1ACC1B0F1ADC177
:10095000B1F1AEC1B2F1AFC1B3F1B0C1B4F1B1C147
:10096000B5F1B2C1B6F1B3C1B7F1B4C1B8F1B5C117
:10097000B9F101015E6B5F6B606B616B9A515E2731
:100980009B515F239C5160239D5161239E515E27A3
:100990009F515F23A0516023A1516123A2515E2783
:1009A000A3515F23A4516023A5516123A6515E2763
:1009B000A7515F23A8516023A9516123AA515E2743
:1009C000AB515F23AC516023AD516123AE515E2723
:1009D000AF515F23B0516023B1516123B2515E2703
:1009E000B3515F23B4516023B5516123B6515E27E3
:1009F000B7515F23B8516023B9516123D8900101E9
:100A0000613360335F335E33D8900101613360330B
:100A10005F335E33D8900101613360335F335E33FF
:100A200000C10CF101C10DF102C10EF103C10FF1C2
:100A300004C110F105C111F106C112F107C113F192
:100A400008C114F109C115F10AC116F10BC117F162
:100A500034C135F111B838EF05F00101620E046FB1
:100A6000010E056F000E066F000E076F41EF05F0D7
:100A70000101A70E046F020E056F000E066F000E37
:100A8000076F5EC100F15FC101F160C102F161C198
:100A900003F1F5EC39F003BF04D01CBE02D01CA05A
:100AA000108C11A059EF05F010BA59EF05F00F8026
:100AB000108A0CC100F10DC101F10EC102F10FC18C
:100AC00003F110C104F111C105F112C106F113C106
:100AD00007F114C108F115C109F116C10AF117C1D6
:100AE0000BF135C134F1EBEF0BF00392ABB2AB98E5
:100AF000AB88030103EE00F080517F0BE92604C0B0
:100B0000EFFF802B8151805D700BD8A48B82000099
:100B10008051815D700BD8A48B9281518019D8B41B
:100B20000790EBEF0BF0F2940101453FEBEF0BF078
:100B3000462BEBEF0BF09E900101533FEBEF0BF0D8
:100B4000542BEBEF0BF09E9211B895EF08F00400D8
:100B500066A1ABEF05F08BB4B5EF05F010ACB5EFC7
:100B600005F08B84109CB6EF05F08B9407B408EF6A
:100B700006F007B008EF06F01EC620F61FC621F6E5
:100B80001CC61EF61DC61FF61AC61CF61BC61DF691
:100B900006C608F607C609F604C606F605C607F631
:100BA00002C604F603C605F626C628F627C629F6A9
:100BB00024C626F625C627F622C624F623C625F621
:100BC0000EC610F60FC611F60CC60EF60DC60FF6C1
:100BD0000AC60CF60BC60DF62EC630F62FC631F639
:100BE0002CC62EF62DC62FF62AC62CF62BC62DF6B1
:100BF00016C618F617C619F614C616F615C617F651
:100C000012C614F613C615F609EC3CF0B7EC3BF02F
:100C1000077C07AC23EF06F0C274C2B41DEF06F0E8
:100C2000C3CFB7F5C4CFB8F50501D890B833B73303
:100C3000D890B833B73324EF06F0C3CF55F1C4CF03
:100C400056F124EF06F0C28207B496EF06F047C1D2
:100C50004BF148C14CF149C14DF14AC14EF15EC161
:100C600062F15FC163F160C164F161C165F113A814
:100C70003CEF06F0138C13989AC1BAF19BC1BBF1FB
:100C80009CC1BCF19DC1BDF19EC1BEF19FC1BFF130
:100C9000A0C1C0F1A1C1C1F1A2C1C2F1A3C1C3F100
:100CA000A4C1C4F1A5C1C5F1A6C1C6F1A7C1C7F1D0
:100CB000A8C1C8F1A9C1C9F1AAC1CAF1ABC1CBF1A0
:100CC000ACC1CCF1ADC1CDF1AEC1CEF1AFC1CFF170
:100CD000B0C1D0F1B1C1D1F1B2C1D2F1B3C1D3F140
:100CE000B4C1D4F1B5C1D5F1B6C1D6F1B7C1D7F110
:100CF000B8C1D8F1B9C1D9F1B7C5B9F5B8C5BAF518
:100D0000B9C5BBF5BAC5BCF5010155515B275651B4
:100D10005C23E86A5D230E2E96EF06F05CC157F166
:100D20005DC158F15B6B5C6B5D6B078E0201002F40
:100D3000EBEF0BF03C0E006F1D50E00BE00AE86695
:100D400012881BBE02D01BB4108E00C10CF101C171
:100D50000DF102C10EF103C10FF104C110F105C183
:100D600011F106C112F107C113F108C114F109C153
:100D700015F10AC116F10BC117F134C135F181AA81
:100D8000FEEF06F015A449EF07F005012F51000A08
:100D9000D8B48CEF07F005012F51010AD8B408EF41
:100DA00007F005012F51020AD8B449EF07F00501F9
:100DB0002F51030AD8B449EF07F005012F51040A57
:100DC000D8B449EF07F005012F51050AD8B449EF0F
:100DD00007F005012F51060AD8B449EF07F00501C5
:100DE0002F51070AD8B449EF07F005012F51320AF5
:100DF000D8B406EF07F02F6B8CEF07F00001165008
:100E0000030AD8B449EF07F08CEF07F08CEF07F036
:100E10000501576713EF07F0586713EF07F059679D
:100E200013EF07F05A6717EF07F08CEF07F05BC579
:100E300000F15CC501F15DC502F15EC503F1010180
:100E4000010E046F000E056F000E066F000E076F97
:100E5000F5EC39F000C15BF501C15CF502C15DF54F
:100E600003C15EF5010100673DEF07F001673DEF4B
:100E700007F002673DEF07F003678CEF07F057C5F7
:100E80005BF558C55CF559C55DF55AC55EF576EF5D
:100E900007F00FBE5EEF07F010A063EF07F001014F
:100EA00047675AEF07F048675AEF07F049675AEF6C
:100EB00007F04A675EEF07F063EF07F007AE63EFF6
:100EC00007F076EF07F00501312F8CEF07F03C0EAD
:100ED000316F302F8CEF07F00101000E626FE00ED2
:100EE000636FA50E646F010E656F138800011650C5
:100EF000000AD8B484EF07F000011650030AD8B4F2
:100F000089EF07F08CEF07F00001010E166E8CEFF1
:100F100007F00001040E166E0501666B37B792EFFD
:100F200007F066810CC100F10DC101F10EC102F1A3
:100F30000FC103F110C104F111C105F112C106F195
:100F400013C107F114C108F115C109F116C10AF165
:100F500017C10BF135C134F100C10CF101C10DF124
:100F600002C10EF103C10FF104C110F105C111F16D
:100F700006C112F107C113F108C114F109C115F13D
:100F80000AC116F10BC117F134C135F101018E67A9
:100F9000D1EF07F08F67D1EF07F09067D1EF07F03F
:100FA0009167D5EF07F006EF08F092C100F193C109
:100FB00001F194C102F195C103F10101010E046F29
:100FC000000E056F000E066F000E076FF5EC39F08E
:100FD00000C192F101C193F102C194F103C195F1F5
:100FE00001010067FBEF07F00167FBEF07F0026705
:100FF000FBEF07F0036706EF08F08EC192F18FC197
:1010000093F190C194F191C195F10F80D57ED5BE39
:101010006ED0D6CF47F1D7CF48F145C149F1E86A44
:10102000E8CF4AF1138A1CBE02D01CA0108C10908D
:1010300047C100F148C101F149C102F14AC103F1C0
:1010400001010A0E046F000E056F000E066F000E00
:10105000076FF5EC39F003AF1080010154A73DEFA5
:1010600008F00F9A0F9C0F9E0101000E5E6F600E3C
:101070005F6F3D0E606F080E616F010147BF4DEF5E
:1010800008F048674DEF08F049674DEF08F04A67F0
:101090004DEF08F0F28872EF08F0F2985E6B5F6B2C
:1010A000606B616B9A6B9B6B9C6B9D6B9E6B9F6B7C
:1010B000A06BA16BA26BA36BA46BA56BA66BA76BBC
:1010C000A86BA96BAA6BAB6BAC6BAD6BAE6BAF6B6C
:1010D000B06BB16BB26BB36BB46BB56BB66BB76B1C
:1010E000B86BB96BD76AD66A0101456B466B0CC108
:1010F00000F10DC101F10EC102F10FC103F110C1E8
:1011000004F111C105F112C106F113C107F114C1B7
:1011100008F115C109F116C10AF117C10BF135C16A
:1011200034F1EBEF0BF0EBEF0BF00201002FFDEFD2
:101130000AF0D59ED6CF47F1D7CF48F145C149F146
:10114000E86AE8CF4AF1138AD76AD66A0101456B8B
:10115000466BD58E1D50E00BE00AE86612881BBE78
:1011600002D01BB4108E1AAE1F8C00C10CF101C14D
:101170000DF102C10EF103C10FF104C110F105C15F
:1011800011F106C112F107C113F108C114F109C12F
:1011900015F10AC116F10BC117F134C135F10FA0D9
:1011A000109A11B8DFEF08F00101620E046F010E12
:1011B000056F000E066F000E076FE8EF08F00101E3
:1011C000A70E046F020E056F000E066F000E076F6C
:1011D00047C100F148C101F149C102F14AC103F11F
:1011E000F5EC39F003BFFBEF08F01CBE02D01CA0E9
:1011F000108C11B00F800CC100F10DC101F10EC1B6
:1012000002F10FC103F110C104F111C105F112C1C6
:1012100006F113C107F114C108F115C109F116C196
:101220000AF117C10BF135C134F102013C0E006F18
:1012300000C10CF101C10DF102C10EF103C10FF1AA
:1012400004C110F105C111F106C112F107C113F17A
:1012500008C114F109C115F10AC116F10BC117F14A
:1012600034C135F181BA38EF09F015B277EF09F0E2
:1012700015A077EF09F015A4C2EF09F005012F5171
:10128000000AD8B405EF0AF005012F51010AD8B4BD
:1012900081EF09F005012F51020AD8B4C2EF09F01D
:1012A00005012F51030AD8B4C2EF09F005012F51EF
:1012B000040AD8B4C2EF09F005012F51050AD8B4C9
:1012C000C2EF09F005012F51060AD8B4C2EF09F0A8
:1012D00005012F51070AD8B4C2EF09F005012F51BB
:1012E000320AD8B47FEF09F02F6B05EF0AF0000146
:1012F0001650030AD8B4C2EF09F005EF0AF005EF63
:101300000AF0050157678CEF09F058678CEF09F078
:1013100059678CEF09F05A6790EF09F005EF0AF072
:101320005BC500F15CC501F15DC502F15EC503F16D
:101330000101010E046F000E056F000E066F000E16
:10134000076FF5EC39F000C15BF501C15CF502C136
:101350005DF503C15EF501010067B6EF09F00167B5
:10136000B6EF09F00267B6EF09F0036705EF0AF080
:1013700057C55BF558C55CF559C55DF55AC55EF5B1
:10138000EFEF09F00FBED7EF09F010A0DCEF09F086
:1013900001014767D3EF09F04867D3EF09F04967C8
:1013A000D3EF09F04A67D7EF09F0DCEF09F007AE99
:1013B000DCEF09F0EFEF09F00501312F05EF0AF03E
:1013C0003C0E316F302F05EF0AF00101000E626F05
:1013D000E00E636FA50E646F010E656F1388000148
:1013E0001650000AD8B4FDEF09F000011650030AA8
:1013F000D8B402EF0AF005EF0AF00001010E166EF4
:1014000005EF0AF00001040E166E0501666B37B792
:101410000BEF0AF066810CC100F10DC101F10EC1A4
:1014200002F10FC103F110C104F111C105F112C1A4
:1014300006F113C107F114C108F115C109F116C174
:101440000AF117C10BF135C134F100C10CF101C132
:101450000DF102C10EF103C10FF104C110F105C17C
:1014600011F106C112F107C113F108C114F109C14C
:1014700015F10AC116F10BC117F134C135F10101A3
:101480008E674AEF0AF08F674AEF0AF090674AEFDB
:101490000AF091674EEF0AF07FEF0AF092C100F177
:1014A00093C101F194C102F195C103F10101010E53
:1014B000046F000E056F000E066F000E076FF5EC4F
:1014C00039F000C192F101C193F102C194F103C15D
:1014D00095F10101006774EF0AF0016774EF0AF0FB
:1014E000026774EF0AF003677FEF0AF08EC192F192
:1014F0008FC193F190C194F191C195F10F8010903B
:1015000047C100F148C101F149C102F14AC103F1EB
:1015100001010A0E046F000E056F000E066F000E2B
:10152000076FF5EC39F003AF1080010154A7A5EF68
:101530000AF00F9A0F9C0F9E0101000E5E6F600E65
:101540005F6F3D0E606F080E616F47C100F148C1CB
:1015500001F149C102F14AC103F10101140E046F06
:10156000050E056F000E066F000E076FF5EC39F0E3
:1015700003AFBEEF0AF0F288E3EF0AF0F2985E6B79
:101580005F6B606B616B9A6B9B6B9C6B9D6B9E6BD7
:101590009F6BA06BA16BA26BA36BA46BA56BA66BDF
:1015A000A76BA86BA96BAA6BAB6BAC6BAD6BAE6B8F
:1015B000AF6BB06BB16BB26BB36BB46BB56BB66B3F
:1015C000B76BB86BB96B0CC100F10DC101F10EC165
:1015D00002F10FC103F110C104F111C105F112C1F3
:1015E00006F113C107F114C108F115C109F116C1C3
:1015F0000AF117C10BF135C134F104008BB408EFC7
:101600000BF010AC08EF0BF08B84109C09EF0BF083
:101610008B9407B45BEF0BF007B05BEF0BF01EC6CB
:1016200020F61FC621F61CC61EF61DC61FF61AC6DA
:101630001CF61BC61DF606C608F607C609F604C644
:1016400006F605C607F602C604F603C605F626C664
:1016500028F627C629F624C626F625C627F622C66A
:1016600024F623C625F60EC610F60FC611F60CC6D4
:101670000EF60DC60FF60AC60CF60BC60DF62EC6F4
:1016800030F62FC631F62CC62EF62DC62FF62AC6FA
:101690002CF62BC62DF616C618F617C619F614C664
:1016A00016F615C617F612C614F613C615F609EC8B
:1016B0003CF0B7EC3BF0077C07AC76EF0BF0C27464
:1016C000C2B470EF0BF0C3CFB7F5C4CFB8F50501C6
:1016D000D890B833B733D890B833B73377EF0BF02F
:1016E000C3CF55F1C4CF56F177EF0BF0C28207B4E8
:1016F000E9EF0BF047C14BF148C14CF149C14DF145
:101700004AC14EF15EC162F15FC163F160C164F133
:1017100061C165F113A88FEF0BF0138C13989AC178
:10172000BAF19BC1BBF19CC1BCF19DC1BDF19EC191
:10173000BEF19FC1BFF1A0C1C0F1A1C1C1F1A2C161
:10174000C2F1A3C1C3F1A4C1C4F1A5C1C5F1A6C131
:10175000C6F1A7C1C7F1A8C1C8F1A9C1C9F1AAC101
:10176000CAF1ABC1CBF1ACC1CCF1ADC1CDF1AEC1D1
:10177000CEF1AFC1CFF1B0C1D0F1B1C1D1F1B2C1A1
:10178000D2F1B3C1D3F1B4C1D4F1B5C1D5F1B6C171
:10179000D6F1B7C1D7F1B8C1D8F1B9C1D9F1B7C540
:1017A000B9F5B8C5BAF5B9C5BBF5BAC5BCF50101FF
:1017B00055515B2756515C23E86A5D230E2EE9EFF5
:1017C0000BF05CC157F15DC158F15B6B5C6B5D6BFD
:1017D000078EEBEF0BF002C0E0FF005001C0D8FF16
:1017E0001000A6B2F1EF0BF00CC0A9FF0BC0A8FFD0
:1017F000A69EA69CA684F29E550EA76EAA0EA76E64
:10180000A682F28EA694A6B203EF0CF00C2A120068
:10181000A96EA69EA69CA680A8500C2A12000401C0
:101820002C0E826F70EC0FF00AEC3BF00C5008ECC1
:101830000CF0E8CF00F10C5008EC0CF0E8CF01F10F
:1018400001AF28EF0CF00101FF0E026FFF0E036FD6
:1018500093EC3AF0296734EF0CF00401200E826F0C
:1018600070EC0FF039EF0CF004012D0E826F70EC6C
:101870000FF09DEC38F0120015941596076A0F6A68
:10188000106A116A126A136A166A0F010D0EC16E90
:10189000860EC06E030EC26E0F01680E896E130EA7
:1018A000926E080E8A6E8A6AF30E936E8B6A900EA1
:1018B000946EC80E08EC0CF0E8CFE8FF1098E8A092
:1018C000108810A805D00E0E256E8E0E266E04D040
:1018D0000F0E256E8F0E266EDAEC3CF025EC3EF0F6
:1018E000F18EF19EFC0E08EC0CF0E8CF0BF00BA093
:1018F00011800BA211820BA411840BA81188C90EB0
:1019000008EC0CF0E8CF1AF0CA0E08EC0CF0E8CFA7
:101910001BF0CB0E08EC0CF0E8CF1CF0CC0E08EC62
:101920000CF0E8CF1DF0FB0E08EC0CF0E8CF37F020
:10193000CE0E08EC0CF0E8CF14F0CD0E08EC0CF055
:10194000E8CF36F01F6A206A0E6A01015B6B5C6BA0
:101950005D6B576B586BF29A0101476B486B496B93
:101960004A6B4B6B4C6B4D6B4E6B4F6B506B516BB3
:10197000526B456B466BD76AD66A0F01280ED56E3F
:10198000F28A9D90B00ECD6E01015E6B5F6B606B55
:10199000616B626B636B646B656B666B676B686BCB
:1019A000696B536B546BCF6ACE6A0F9A0F9C0F9E74
:1019B0009D80760ECA6E9D8202013C0E006FCC6A3D
:1019C000160E08EC0CF0E8CF00F1170E08EC0CF046
:1019D000E8CF01F1180E08EC0CF0E8CF02F1190E77
:1019E00008EC0CF0E8CF03F1010103AF12EF0DF0AA
:1019F0000AEC3BF0160E0C6E00C10BF0F1EC0BF094
:101A0000170E0C6E01C10BF0F1EC0BF0180E0C6E02
:101A100002C10BF0F1EC0BF0190E0C6E03C10BF0D0
:101A2000F1EC0BF000C18EF101C18FF102C190F118
:101A300003C191F100C192F101C193F102C194F18E
:101A400003C195F11A0E08EC0CF0E8CF00F11B0E63
:101A500008EC0CF0E8CF01F11C0E08EC0CF0E8CF1C
:101A600002F11D0E08EC0CF0E8CF03F1010103AF09
:101A700068EF0DF00AEC3BF01A0E0C6E00C10BF093
:101A8000F1EC0BF01B0E0C6E01C10BF0F1EC0BF046
:101A90001C0E0C6E02C10BF0F1EC0BF01D0E0C6E67
:101AA00003C10BF0F1EC0BF01A0E08EC0CF0E8CFD0
:101AB00000F11B0E08EC0CF0E8CF01F11C0E08EC55
:101AC0000CF0E8CF02F11D0E08EC0CF0E8CF03F1AA
:101AD00000C196F101C197F102C198F103C199F1DA
:101AE000240EAC6E900EAB6E240EAC6E080EB86E6B
:101AF000000EB06E1F0EAF6E0401806B816B0F0184
:101B0000900EAB6E0F019D8A0301806B816BC26BDF
:101B10008B927FEC41F07FEC41F0880E08EC0CF0EA
:101B2000E8CF00F1890E08EC0CF0E8CF01F10101DB
:101B300001AFB3EF0DF00AEC3BF0880E0C6E00C164
:101B40000BF0F1EC0BF0890E0C6E01C10BF0F1EC17
:101B50000BF0880E08EC0CF0E8CF00F1890E08ECD1
:101B60000CF0E8CF01F100C140F601C141F602C11D
:101B700042F603C143F65DEC45F05DEC3FF0200E0C
:101B800008EC0CF0E8CF2FF505012F51FF0AD8A47F
:101B9000D1EF0DF02F6B200E0C6E2FC50BF0F1EC7A
:101BA0000BF00501010E306F3C0E316F250E08EC75
:101BB0000CF0E8CF00F1260E08EC0CF0E8CF01F1B4
:101BC000270E08EC0CF0E8CF02F1280E08EC0CF020
:101BD000E8CF03F1010103AF08EF0EF00AEC3BF090
:101BE000250E0C6E00C10BF0F1EC0BF0260E0C6E06
:101BF00001C10BF0F1EC0BF0270E0C6E02C10BF0E3
:101C0000F1EC0BF0280E0C6E03C10BF0F1EC0BF0B5
:101C100000C157F501C158F502C159F503C15AF584
:101C200000C15BF501C15CF502C15DF503C15EF564
:101C3000290E08EC0CF0E8CF5FF5050160515F5DFF
:101C4000D8A05FC560F5210E08EC0CF0E8CF00F1DC
:101C5000220E08EC0CF0E8CF01F1230E08EC0CF09A
:101C6000E8CF02F1240E08EC0CF0E8CF03F10101FB
:101C700003AF69EF0EF00AEC3BF0210E0C6E00C1D1
:101C80000BF0F1EC0BF0220E0C6E01C10BF0F1EC3D
:101C90000BF0230E0C6E02C10BF0F1EC0BF0240ED6
:101CA0000C6E03C10BF0F1EC0BF0210E08EC0CF004
:101CB000E8CF00F1220E08EC0CF0E8CF01F1230E82
:101CC00008EC0CF0E8CF02F1240E08EC0CF0E8CFA1
:101CD00003F100C161F501C162F502C163F503C101
:101CE00064F5A5EC3EF08BEC3DF0E3EC3CF0159098
:101CF000C70E08EC0CF0E8CF00F1010100B184EF51
:101D00000EF0159285EF0EF0158281AA93EF0EF07A
:101D100015B48EEF0EF0158093EF0EF09CEC45F0AD
:101D200015A003EF46F05BEC3CF007900001F28E4B
:101D3000F28C12AE03D012BC1CEF21F007B02FEFD3
:101D400036F00FB02BEF2FF010BE2BEF2FF012B8A4
:101D50002BEF2FF000011650010AD8B424EF27F022
:101D600081BABBEF0EF000011650040AD8B4C8EFD8
:101D700023F0C1EF0EF000011650040AD8B460EF52
:101D800027F00301805181197F0BD8B42FEF36F073
:101D900013EE00F081517F0BE126812BE7CFE8FFA6
:101DA000E00BD8B42FEF36F023EE82F0C2513F0B98
:101DB000D926E7CFDFFFC22BDF50780AD8A42FEF58
:101DC00036F0078092C100F193C101F194C102F194
:101DD00095C103F10101040E046F000E056F000EA2
:101DE000066F000E076FF5EC39F000AF01EF0FF052
:101DF0000101030E926F000E936F000E946F000EA0
:101E0000956F03018251720AD8B4ACEF2EF0825163
:101E1000520AD8B4ACEF2EF08251750AD8B4ACEFA8
:101E20002EF08251680AD8B484EF0FF08251630A11
:101E3000D8B4E9EF32F08251690AD8B46AEF2AF0D7
:101E400082517A0AD8B47DEF2BF08251490AD8B476
:101E500009EF2AF08251500AD8B427EF29F08251B5
:101E6000700AD8B46AEF29F08251540AD8B495EFB9
:101E700029F08251740AD8B4DBEF29F08251410A6B
:101E8000D8B489EF10F082514B0AD8B486EF0FF026
:101E900082516D0AD8B4F9EF14F082514D0AD8B4CA
:101EA00012EF15F08251730AD8B4DCEF2DF0825195
:101EB000530AD8B441EF2EF082514C0AD8B475EFD2
:101EC0001CF08251760AD8B4A1EF15F08251590A5C
:101ED000D8B44AEF14F012AE01D0128C20EF33F0D8
:101EE000040114EE00F080517F0BE12682C4E7FF6D
:101EF000802B120004010D0E826F70EC0FF00A0EA1
:101F0000826F70EC0FF012001EEF33F004014B0EE5
:101F1000826F70EC0FF004012C0E826F70EC0FF0EA
:101F200081B802D036B630D003018351430AD8B409
:101F3000CBEF0FF003018351630AD8B4CDEF0FF05C
:101F400003018351520AD8B4CFEF0FF0030183513C
:101F5000720AD8B4D1EF0FF003018351470AD8B405
:101F6000D3EF0FF003018351670AD8B4D5EF0FF018
:101F700003018351540AD8B4D7EF0FF00301835102
:101F8000740AD8B447EF10F003018351550AD8B44E
:101F9000D9EF0FF083D036807BD0369079D036825F
:101FA00077D0369275D0368473D0369471D0368619
:101FB0006FD084C330F185C331F186C332F187C35A
:101FC00033F10101296B58EC3BF0CFEC3AF000C142
:101FD00004F101C105F102C106F103C107F14BECA7
:101FE0003BF0200EF86EF76AF66A0900F5CF2CF187
:101FF0000900F5CF2DF10900F5CF2EF10900F5CF3D
:102000002FF10900F5CF30F10900F5CF31F10900CA
:10201000F5CF32F10900F5CF33F10101296B58EC0E
:102020003BF0CFEC3AF0F5EC39F00101006720EF1E
:1020300010F0016720EF10F0026720EF10F0036747
:1020400001D025D004014E0E826F70EC0FF0040118
:102050006F0E826F70EC0FF004014D0E826F70EC0A
:102060000FF00401610E826F70EC0FF00401740E2A
:10207000826F70EC0FF00401630E826F70EC0FF052
:102080000401680E826F70EC0FF01EEF33F036968D
:10209000CD0E0C6E36C00BF0F1EC0BF0CD0E08EC53
:1020A0000CF0E8CF36F036B006D00401630E826F34
:1020B00070EC0FF005D00401430E826F70EC0FF04E
:1020C00036B206D00401720E826F70EC0FF005D0AC
:1020D0000401520E826F70EC0FF036B406D004018A
:1020E000670E826F70EC0FF005D00401470E826F0F
:1020F00070EC0FF036B606D00401740E826F70ECEF
:102100000FF005D00401540E826F70EC0FF01EEF3B
:1021100033F00401410E826F70EC0FF00301835124
:10212000310AD8B46AEF13F003018351320AD8B4EC
:102130009AEF12F003018351330AD8B423EF12F05F
:1021400003018351340AD8B413EF11F00301835112
:10215000350AD8B4B3EF10F004013F0E826F70EC73
:102160000FF01EEF33F003018451300AD8B4D9EFD9
:1021700010F003018451310AD8B4DCEF10F00301F0
:102180008451650AD8B4CDEF10F003018451640A7C
:10219000D8B4D0EF10F0DDEF10F03790D1EF10F0A1
:1021A0003780FB0E0C6E37C00BF0F1EC0BF0DDEF5F
:1021B00010F08B90DDEF10F08B800401350E826FF4
:1021C00070EC0FF004012C0E826F70EC0FF08BB0EE
:1021D000F1EF10F00401300E826F70EC0FF0F6EFAB
:1021E00010F00401310E826F70EC0FF004012C0E20
:1021F000826F70EC0FF0FB0E08EC0CF0E8CF37F0BC
:1022000037A00AEF11F00401640E826F70EC0FF03A
:102210000FEF11F00401650E826F70EC0FF011EFFB
:1022200011F01EEF33F0CC0E08EC0CF0E8CF0BF001
:1022300004012C0E826F70EC0FF003018451310AFF
:10224000D8B437EF11F003018451300AD8B439EF14
:1022500011F0030184514D0AD8B443EF11F003018A
:102260008451540AD8B44AEF11F061EF11F08A8416
:1022700001D08A940BAE04D00BAC02D00BBA21D0A3
:10228000E00E0B1218D01F0E0B168539E844E00B38
:102290000B1211D0E00E0B164BEC3BF085C332F164
:1022A00086C333F10101296B58EC3BF0CFEC3AF0D7
:1022B00000511F0B0B12CC0E0C6E0BC00BF0F1EC8F
:1022C0000BF00401340E826F70EC0FF004012C0E41
:1022D000826F70EC0FF0CC0E08EC0CF0E8CF1DF024
:1022E0008AB406D00401300E826F70EC0FF005D076
:1022F0000401310E826F70EC0FF004012C0E826F1E
:1023000070EC0FF01D38E840070BE8CF82F40401B1
:10231000300E822770EC0FF004012C0E826F70ECEF
:102320000FF00AEC3BF01D501F0BE8CF00F193ECCF
:102330003AF032C182F40401300E822770EC0FF0C3
:1023400033C182F40401300E822770EC0FF00401D7
:102350002C0E826F70EC0FF00AEC3BF030C000F1F5
:1023600000AF0BD0FF0E016FFF0E026FFF0E036F69
:1023700004012D0E826F70EC0FF093EC3AF031C136
:1023800082F40401300E822770EC0FF032C182F427
:102390000401300E822770EC0FF033C182F4040187
:1023A000300E822770EC0FF004012C0E826F70EC5F
:1023B0000FF00AEC3BF02FC000F193EC3AF031C182
:1023C00082F40401300E822770EC0FF032C182F4E7
:1023D0000401300E822770EC0FF033C182F4040147
:1023E000300E822770EC0FF004012C0E826F70EC1F
:1023F0000FF00AEC3BF031C000F100AF0BD0FF0E44
:10240000016FFF0E026FFF0E036F04012D0E826F2E
:1024100070EC0FF093EC3AF031C182F40401300E0D
:10242000822770EC0FF032C182F40401300E822753
:1024300070EC0FF033C182F40401300E822770EC8F
:102440000FF01EEF33F0CB0E08EC0CF0E8CF0BF0E2
:1024500004012C0E826F70EC0FF003018451450AC9
:10246000D8B447EF12F003018451440AD8B44AEFBC
:1024700012F003018451300AD8B44DEF12F0030179
:102480008451310AD8B451EF12F05CEF12F00B9E78
:1024900056EF12F00B8E56EF12F0FC0E0B1656EFA5
:1024A00012F0FC0E0B160B8056EF12F0CB0E0C6EDA
:1024B0000BC00BF0F1EC0BF00401330E826F70ECEB
:1024C0000FF004012C0E826F70EC0FF0CB0E08ECB5
:1024D0000CF0E8CF1CF01CBE75EF12F00401450EA5
:1024E000826F70EC0FF07AEF12F00401440E826FED
:1024F00070EC0FF004012C0E826F70EC0FF00401F1
:10250000300E826F70EC0FF004012C0E826F70ECB5
:102510000FF01CB093EF12F00401300E826F70ECDC
:102520000FF098EF12F00401310E826F70EC0FF093
:102530001EEF33F0CA0E08EC0CF0E8CF0BF00401EC
:102540002C0E826F70EC0FF003018451450AD8B451
:10255000D6EF12F003018451440AD8B4D9EF12F037
:10256000030184514D0AD8B4E2EF12F00301845103
:10257000410AD8B4DCEF12F003018451460AD8B402
:10258000DFEF12F003018451560AD8B4EAEF12F0DB
:1025900003018451500AD8B4F5EF12F003018451BD
:1025A000520AD8B4F8EF12F001EF13F00B9EFBEFD4
:1025B00012F00B8EFBEF12F00B9CFBEF12F00B8C6A
:1025C000FBEF12F0FC0E0B1685C3E8FF030B0B129A
:1025D000FBEF12F0C70E0B1685C3E8FF070BE846AA
:1025E000E846E8460B12FBEF12F00B84FBEF12F00B
:1025F0000B94FBEF12F0CA0E0C6E0BC00BF0F1EC5B
:102600000BF0CA0E08EC0CF0E8CF1BF00401320E00
:10261000826F70EC0FF004012C0E826F70EC0FF0E3
:102620001BBE1AEF13F00401450E826F70EC0FF021
:102630001FEF13F00401440E826F70EC0FF00401E1
:102640002C0E826F70EC0FF01BC0E8FF030BE8CF7D
:1026500082F40401300E822770EC0FF004012C0E7E
:10266000826F70EC0FF01BBC3DEF13F00401410EC4
:10267000826F70EC0FF042EF13F00401460E826F90
:1026800070EC0FF004012C0E826F70EC0FF01BC089
:10269000E8FF380BE842E842E842E8CF82F4040160
:1026A000300E822770EC0FF004012C0E826F70EC5C
:1026B0000FF01BB463EF13F00401520E826F70EC45
:1026C0000FF068EF13F00401500E826F70EC0FF002
:1026D0001EEF33F0C90E08EC0CF0E8CF0BF004014C
:1026E0002C0E826F70EC0FF003018451450AD8B4B0
:1026F00088EF13F003018451440AD8B48BEF13F030
:10270000030184514D0AD8B48EEF13F09CEF13F0FF
:102710000B9E96EF13F00B8E96EF13F0F80E0B1640
:1027200085C3E8FF070B0B1296EF13F0C90E0C6E72
:102730000BC00BF0F1EC0BF00401310E826F70EC6A
:102740000FF004012C0E826F70EC0FF0C90E08EC34
:102750000CF0E8CF1AF01ABE06D00401450E826FC5
:1027600070EC0FF005D00401440E826F70EC0FF096
:1027700004012C0E826F70EC0FF01AC0E8FF070BFB
:10278000E8CF82F40401300E822770EC0FF00401D0
:102790002C0E826F70EC0FF007800AEC3BF02BC020
:1027A000E8FF003B00430043030B93EC3AF033C1D6
:1027B00082F40401300E822770EC0FF004012C0E1D
:1027C000826F70EC0FF00AEC3BF02BC001F1019F1F
:1027D000019D2CC000F1010193EC3AF02FC182F46D
:1027E0000401300E822770EC0FF030C182F4040136
:1027F000300E822770EC0FF031C182F40401300EEC
:10280000822770EC0FF032C182F40401300E82276F
:1028100070EC0FF033C182F40401300E822770ECAB
:102820000FF004012C0E826F70EC0FF00AEC3BF0FD
:102830002DC001F12EC000F1D89001330033D890A3
:1028400001330033010193EC3AF02FC182F404010B
:10285000300E822770EC0FF030C182F40401300E8C
:10286000822770EC0FF031C182F40401300E822710
:1028700070EC0FF032C182F40401300E822770EC4C
:102880000FF033C182F40401300E822770EC0FF098
:102890001EEF33F0FC0E08EC0CF0E8CF0BF0030158
:1028A0008351520AD8B481EF14F003018351720AA4
:1028B000D8B484EF14F003018351500AD8B487EFE1
:1028C00014F003018351700AD8B48AEF14F00301A5
:1028D0008351550AD8B48DEF14F003018351750A62
:1028E000D8B490EF14F003018351430AD8B499EFA0
:1028F00014F003018351630AD8B49CEF14F0A5EFE0
:1029000014F00B909FEF14F00B809FEF14F00B92DC
:102910009FEF14F00B829FEF14F00B949FEF14F0D5
:102920000B849FEF14F00B969FEF14F00B869FEF34
:1029300014F00B989FEF14F00B889FEF14F0FC0E2F
:102940000C6E0BC00BF0F1EC0BF00401590E826F12
:1029500070EC0FF01190119211941198FC0E08EC8C
:102960000CF0E8CF0BF00BA011800BA211820BA48E
:1029700011840BA8118811A0C5EF14F00401520EA8
:10298000826F70EC0FF0CAEF14F00401720E826FC8
:1029900070EC0FF011A8D4EF14F00401430E826F15
:1029A00070EC0FF0D9EF14F00401630E826F70EC3D
:1029B0000FF011A2E3EF14F00401500E826F70ECDF
:1029C0000FF0E8EF14F00401700E826F70EC0FF05E
:1029D00011A4F2EF14F00401550E826F70EC0FF0A9
:1029E000F7EF14F00401750E826F70EC0FF01EEF1C
:1029F00033F004016D0E826F70EC0FF00301835110
:102A0000300AD8B451EF15F003018351310AD8B41C
:102A100064EF15F003018351320AD8B477EF15F053
:102A200020EF33F004014D0E826F70EC0FF04BEC91
:102A30003BF084C331F185C332F186C333F1010128
:102A4000296B58EC3BF0CFEC3AF003018351300A8C
:102A5000D8B439EF15F003018351310AD8B441EFEE
:102A600015F003018351320AD8B449EF15F020EF75
:102A700033F0FD0E0C6E00C10BF0F1EC0BF051EFDA
:102A800015F0FE0E0C6E00C10BF0F1EC0BF064EFD4
:102A900015F0FF0E0C6E00C10BF0F1EC0BF077EFB0
:102AA00015F00401300E826F70EC0FF004012C0E53
:102AB000826F70EC0FF00AEC3BF0FD0E08EC0CF0AE
:102AC000E8CF00F188EF15F00401310E826F70EC51
:102AD0000FF004012C0E826F70EC0FF00AEC3BF04B
:102AE000FE0E08EC0CF0E8CF00F188EF15F00401C1
:102AF000320E826F70EC0FF00AEC3BF004012C0EEA
:102B0000826F70EC0FF0FF0E08EC0CF0E8CF00F1D4
:102B100093EC3AF031C182F40401300E822770EC5C
:102B20000FF032C182F40401300E822770EC0FF0F6
:102B300033C182F40401300E822770EC0FF01EEFD7
:102B400033F003018351300AD8B446EF17F0030184
:102B50008351310AD8B47DEF17F003018351320A53
:102B6000D8B432EF19F003018351330AD8B4E7EF38
:102B70001AF003018351340AD8B48DEF1BF003011E
:102B80008351730AD8B428EF16F003018351760AF3
:102B9000D8B42AEF16F003018351740AD8B415EFA4
:102BA00016F003018351540AD8B4DAEF15F0D8A413
:102BB00020EF33F00401760E826F70EC0FF0040109
:102BC000540E826F70EC0FF007840001880E0C6EBB
:102BD0004BEC3BF02981030184512D0AD8B4F3EF6B
:102BE00015F00101299185C32FF186C330F187C308
:102BF00031F188C332F189C333F158EC3BF0CFECAB
:102C00003AF000C10BF0F1EC0BF001C10BF0F1EC6C
:102C10000BF0880E08EC0CF0E8CF40F6890E08ECBB
:102C20000CF0E8CF41F620EF16F00401760E826F2B
:102C300070EC0FF00401740E826F70EC0FF00784DB
:102C40000001880E0C6E0FEC0CF00794D4EF27F007
:102C500028EC16F00401760E826F70EC0FF0040180
:102C6000760E826F70EC0FF007844DEC37F00401A4
:102C70002C0E826F70EC0FF00101036B026B3BC6F0
:102C800001F13AC600F101AF4BEF16F00101FF0E62
:102C9000026FFF0E036F93EC3AF0296752EF16F0C4
:102CA00057EF16F004012D0E826F70EC0FF02FC15C
:102CB00082F40401300E822770EC0FF030C182F4F0
:102CC0000401300E822770EC0FF031C182F4040150
:102CD000300E822770EC0FF032C182F40401300E06
:102CE000822770EC0FF033C182F40401300E82278A
:102CF00070EC0FF004012C0E826F70EC0FF00101EC
:102D0000036B026B3DC601F13CC600F101AF8EEFD3
:102D100016F00101FF0E026FFF0E036F93EC3AF005
:102D2000296795EF16F09AEF16F004012D0E826FC9
:102D300070EC0FF02FC182F40401300E822770EC8A
:102D40000FF030C182F40401300E822770EC0FF0D6
:102D500031C182F40401300E822770EC0FF032C1D1
:102D600082F40401300E822770EC0FF033C182F43C
:102D70000401300E822770EC0FF004012C0E826FDC
:102D800070EC0FF00101036B026B3FC601F13EC610
:102D900000F101AFD1EF16F00101FF0E026FFF0E3F
:102DA000036F93EC3AF02967D8EF16F0DDEF16F0D9
:102DB00004012D0E826F70EC0FF02FC182F404011C
:102DC000300E822770EC0FF030C182F40401300E17
:102DD000822770EC0FF031C182F40401300E82279B
:102DE00070EC0FF032C182F40401300E822770ECD7
:102DF0000FF033C182F40401300E822770EC0FF023
:102E000004012C0E826F70EC0FF00101036B026B5A
:102E100037C601F136C600F101AF14EF17F001011A
:102E2000FF0E026FFF0E036F93EC3AF029671BEF62
:102E300017F020EF17F004012D0E826F70EC0FF0E9
:102E40002FC182F40401300E822770EC0FF030C1E4
:102E500082F40401300E822770EC0FF031C182F44D
:102E60000401300E822770EC0FF032C182F40401AD
:102E7000300E822770EC0FF033C182F40401300E63
:102E8000822770EC0FF00794D4EF27F00401760E40
:102E9000826F70EC0FF00401300E826F70EC0FF057
:102EA00004012C0E826F70EC0FF091EC3BF00AECF9
:102EB0003BF000C600F101C601F193EC3AF030C1DD
:102EC00082F40401300E822770EC0FF031C182F4DD
:102ED0000401300E822770EC0FF032C182F404013D
:102EE000300E822770EC0FF033C182F40401300EF3
:102EF000822770EC0FF0D4EF27F00401760E826F7A
:102F000070EC0FF00401310E826F70EC0FF007844B
:102F10000101036B026B02C600F103C601F101AFB0
:102F200096EF17F0FF0E026FFF0E036F0101076BA4
:102F3000066B04C604F105C605F105AFA4EF17F052
:102F4000FF0E066FFF0E076FFAEC39F00101076BF9
:102F5000066B06C604F107C605F105AFB4EF17F01E
:102F6000FF0E066FFF0E076FFAEC39F00101076BD9
:102F7000066B08C604F109C605F105AFC4EF17F0EA
:102F8000FF0E066FFF0E076FFAEC39F0D8900101C3
:102F90000333023301330033D8900101033302338A
:102FA0000133003304012C0E826F70EC0FF001012D
:102FB000036B026B01C101F100C100F101AFE6EF4B
:102FC00017F00101FF0E026FFF0E036F93EC3AF052
:102FD0002967EDEF17F0F2EF17F004012D0E826F65
:102FE00070EC0FF02FC182F40401300E822770ECD8
:102FF0000FF030C182F40401300E822770EC0FF024
:1030000031C182F40401300E822770EC0FF032C11E
:1030100082F40401300E822770EC0FF033C182F489
:103020000401300E822770EC0FF00101036B026B7C
:103030000AC600F10BC601F101AF23EF18F0FF0E35
:10304000026FFF0E036F0101076B066B0CC604F1E4
:103050000DC605F105AF31EF18F0FF0E066FFF0E3C
:10306000076FFAEC39F00101076B066B0EC604F12D
:103070000FC605F105AF41EF18F0FF0E066FFF0E0A
:10308000076FFAEC39F00101076B066B10C604F10B
:1030900011C605F105AF51EF18F0FF0E066FFF0ED8
:1030A000076FFAEC39F0D890010103330233013392
:1030B0000033D8900101033302330133003304019C
:1030C0002C0E826F70EC0FF00101036B026B01C1DB
:1030D00001F100C100F101AF73EF18F00101FF0E23
:1030E000026FFF0E036F93EC3AF029677AEF18F046
:1030F0007FEF18F004012D0E826F70EC0FF02FC1DE
:1031000082F40401300E822770EC0FF030C182F49B
:103110000401300E822770EC0FF031C182F40401FB
:10312000300E822770EC0FF032C182F40401300EB1
:10313000822770EC0FF033C182F40401300E822735
:1031400070EC0FF00101036B026B12C600F113C6A5
:1031500001F101AFB0EF18F0FF0E026FFF0E036F29
:103160000101076B066B14C604F115C605F105AF26
:10317000BEEF18F0FF0E066FFF0E076FFAEC39F086
:103180000101076B066B16C604F117C605F105AF02
:10319000CEEF18F0FF0E066FFF0E076FFAEC39F056
:1031A0000101076B066B18C604F119C605F105AFDE
:1031B000DEEF18F0FF0E066FFF0E076FFAEC39F026
:1031C000D89001010333023301330033D890010159
:1031D000033302330133003304012C0E826F70EC91
:1031E0000FF00101036B026B01C101F100C100F19D
:1031F00001AF00EF19F00101FF0E026FFF0E036F28
:1032000093EC3AF0296707EF19F00CEF19F004017D
:103210002D0E826F70EC0FF02FC182F40401300E7E
:10322000822770EC0FF030C182F40401300E822747
:1032300070EC0FF031C182F40401300E822770EC83
:103240000FF032C182F40401300E822770EC0FF0CF
:1032500033C182F40401300E822770EC0FF0079422
:10326000D4EF27F00401760E826F70EC0FF00401AA
:10327000320E826F70EC0FF007840101036B026B5A
:103280001AC600F11BC601F101AF4BEF19F0FF0E9A
:10329000026FFF0E036F0101076B066B1CC604F182
:1032A0001DC605F105AF59EF19F0FF0E066FFF0EB1
:1032B000076FFAEC39F00101076B066B1EC604F1CB
:1032C0001FC605F105AF69EF19F0FF0E066FFF0E7F
:1032D000076FFAEC39F00101076B066B20C604F1A9
:1032E00021C605F105AF79EF19F0FF0E066FFF0E4D
:1032F000076FFAEC39F0D890010103330233013340
:103300000033D89001010333023301330033040149
:103310002C0E826F70EC0FF00101036B026B01C188
:1033200001F100C100F101AF9BEF19F00101FF0EA7
:10333000026FFF0E036F93EC3AF02967A2EF19F0CA
:10334000A7EF19F004012D0E826F70EC0FF02FC162
:1033500082F40401300E822770EC0FF030C182F449
:103360000401300E822770EC0FF031C182F40401A9
:10337000300E822770EC0FF032C182F40401300E5F
:10338000822770EC0FF033C182F40401300E8227E3
:1033900070EC0FF00101036B026B22C600F123C633
:1033A00001F101AFD8EF19F0FF0E026FFF0E036FAE
:1033B0000101076B066B24C604F125C605F105AFB4
:1033C000E6EF19F0FF0E066FFF0E076FFAEC39F00B
:1033D0000101076B066B26C604F127C605F105AF90
:1033E000F6EF19F0FF0E066FFF0E076FFAEC39F0DB
:1033F0000101076B066B28C604F129C605F105AF6C
:1034000006EF1AF0FF0E066FFF0E076FFAEC39F0A9
:10341000D89001010333023301330033D890010106
:10342000033302330133003304012C0E826F70EC3E
:103430000FF00101036B026B01C101F100C100F14A
:1034400001AF28EF1AF00101FF0E026FFF0E036FAC
:1034500093EC3AF029672FEF1AF034EF1AF00401D9
:103460002D0E826F70EC0FF02FC182F40401300E2C
:10347000822770EC0FF030C182F40401300E8227F5
:1034800070EC0FF031C182F40401300E822770EC31
:103490000FF032C182F40401300E822770EC0FF07D
:1034A00033C182F40401300E822770EC0FF0010169
:1034B000036B026B2AC600F12BC601F101AF65EF69
:1034C0001AF0FF0E026FFF0E036F0101076B066B10
:1034D0002CC604F12DC605F105AF73EF1AF0FF0EEF
:1034E000066FFF0E076FFAEC39F00101076B066BF0
:1034F0002EC604F12FC605F105AF83EF1AF0FF0EBB
:10350000066FFF0E076FFAEC39F00101076B066BCF
:1035100030C604F131C605F105AF93EF1AF0FF0E86
:10352000066FFF0E076FFAEC39F0D89001010333F4
:10353000023301330033D8900101033302330133E6
:10354000003304012C0E826F70EC0FF00101036B4D
:10355000026B01C101F100C100F101AFB5EF1AF03A
:103560000101FF0E026FFF0E036F93EC3AF0296723
:10357000BCEF1AF0C1EF1AF004012D0E826F70EC4F
:103580000FF02FC182F40401300E822770EC0FF08F
:1035900030C182F40401300E822770EC0FF031C18B
:1035A00082F40401300E822770EC0FF032C182F4F5
:1035B0000401300E822770EC0FF033C182F4040155
:1035C000300E822770EC0FF00794D4EF27F004013F
:1035D000760E826F70EC0FF00401330E826F70EC88
:1035E0000FF004012C0E826F70EC0FF085C382F493
:1035F00070EC0FF0640E0D6E03018551320A02E18A
:103600006A0E0D6E03018551330A02E1700E0D6ED4
:1036100003018551340A02E1760E0D6E03018551D6
:10362000350A02E17C0E0D6E03018551360A02E176
:10363000820E0D6E03018651780A65E00DC00CF014
:103640004BEC3BF02981030187512D0AD8B42BEFB5
:103650001BF00101299188C32FF189C330F18AC37E
:1036600031F18BC332F18CC333F158EC3BF0CFEC2A
:103670003AF000C10BF0F1EC0BF001C10BF0F1ECF2
:103680000BF04BEC3BF0298103018E512D0AD8B48D
:103690004CEF1BF0010129918FC32FF190C330F142
:1036A00091C331F192C332F193C333F158EC3BF043
:1036B000CFEC3AF000C10BF0F1EC0BF001C10BF0D4
:1036C000F1EC0BF04BEC3BF02981030195512D0AF5
:1036D000D8B46DEF1BF00101299196C32FF197C368
:1036E00030F198C331F199C332F19AC333F158ECF8
:1036F0003BF0CFEC3AF000C10BF0F1EC0BF001C164
:103700000BF0F1EC0BF00DC00CF00FEC0CF00FEC2B
:103710000CF00FEC0CF0D4EF27F00401760E826F62
:1037200070EC0FF00401340E826F70EC0FF00301A7
:103730008451780AD8B465EF1CF03E0E0C6E4BEC49
:103740003BF02981030185512D0AD8B4AAEF1BF063
:103750000101299186C32FF187C330F188C331F16C
:1037600089C332F18AC333F158EC3BF0CFEC3AF025
:1037700000C10BF0F1EC0BF001C10BF0F1EC0BF020
:103780004BEC3BF0298103018C512D0AD8B4CBEFCF
:103790001BF0010129918DC32FF18EC330F18FC32E
:1037A00031F190C332F191C333F158EC3BF0CFECDF
:1037B0003AF000C10BF0F1EC0BF001C10BF0F1ECB1
:1037C0000BF04BEC3BF02981030193512D0AD8B447
:1037D000ECEF1BF00101299194C32FF195C330F157
:1037E00096C331F197C332F198C333F158EC3BF0F3
:1037F000CFEC3AF000C10BF0F1EC0BF001C10BF093
:10380000F1EC0BF04BEC3BF0298103019A512D0AAE
:10381000D8B40DEF1CF0010129919BC32FF19CC37B
:1038200030F19DC331F19EC332F19FC333F158ECA7
:103830003BF0CFEC3AF000C10BF0F1EC0BF001C122
:103840000BF0F1EC0BF04BEC3BF029810301A151A3
:103850002D0AD8B42EEF1CF001012991A2C32FF13B
:10386000A3C330F1A4C331F1A5C332F1A6C333F130
:1038700058EC3BF0CFEC3AF000C10BF0F1EC0BF060
:1038800001C10BF0F1EC0BF04BEC3BF02981030193
:10389000A8512D0AD8B44FEF1CF001012991A9C3FA
:1038A0002FF1AAC330F1ABC331F1ACC332F1ADC3D8
:1038B00033F158EC3BF0CFEC3AF000C10BF0F1ECF7
:1038C0000BF001C10BF0F1EC0BF03E0E0C6E0FECA7
:1038D0000CF00FEC0CF00FEC0CF00FEC0CF00FEC0C
:1038E0000CF00FEC0CF0D4EF27F003018351300AF9
:1038F000D8B4C9EF21F003018351310AD8B4F6EFEF
:1039000022F003018351320AD8B464EF23F003019B
:103910008351330AD8B474EF23F003018351340A7E
:10392000D8B4CFEF23F003018351350AD8B478EF30
:1039300027F003018351360AD8B4A6EF27F003011C
:103940008351370AD8B4A1EF1FF003018351380A1D
:10395000D8B43FEF20F003018351440AD8B4CDEF2F
:103960001DF003018351640AD8B4EDEF1DF003018B
:103970008351460AD8B47DEF26F0030183514D0AE6
:10398000D8B41AEF1EF0030183516D0AD8B434EF96
:103990001EF0030183515A0AD8B470EF22F00301DC
:1039A0008351490AD8B4A6EF28F003018351500A85
:1039B000D8B4D8EF27F003018351540AD8B451EF9B
:1039C00028F003018351630AD8B454EF1EF00301B9
:1039D0008351430AD8B44CEF1FF003018351730A9B
:1039E000D8B452EF1EF003018351610AD8B41AEF24
:1039F0001DF003018351650AD8B419EF22F00301C9
:103A00008351450AD8B427EF22F003018351620A9B
:103A1000D8B435EF22F003018351420AD8B443EF02
:103A200022F003018351760AD8B451EF22F0D8A4D2
:103A300020EF33F004014C0E826F70EC0FF00401A4
:103A4000610E826F70EC0FF08BEC3DF004012C0ED8
:103A5000826F70EC0FF00AEC3BF0AFC500F1010192
:103A600093EC3AF031C182F40401300E822770ECFD
:103A70000FF032C182F40401300E822770EC0FF097
:103A800033C182F40401300E822770EC0FF0040180
:103A90002C0E826F70EC0FF00AEC3BF0B0C500F119
:103AA000010193EC3AF031C182F40401300E822717
:103AB00070EC0FF032C182F40401300E822770ECFA
:103AC0000FF033C182F40401300E822770EC0FF046
:103AD00004012C0E826F70EC0FF00AEC3BF0B1C5C4
:103AE00000F1010193EC3AF031C182F40401300E8F
:103AF000822770EC0FF032C182F40401300E82276D
:103B000070EC0FF033C182F40401300E822770ECA8
:103B10000FF004012C0E826F70EC0FF00AEC3BF0FA
:103B2000B2C500F1010193EC3AF031C182F4040115
:103B3000300E822770EC0FF032C182F40401300E97
:103B4000822770EC0FF033C182F40401300E82271B
:103B500070EC0FF004012C0E826F70EC0FF00AEC89
:103B60003BF0B6C500F1010193EC3AF031C182F4AB
:103B70000401300E822770EC0FF032C182F4040190
:103B8000300E822770EC0FF033C182F40401300E46
:103B9000822770EC0FF0D4EF27F003018451300A34
:103BA000D8B4D9EF1DF003018451310AD8B4DDEF48
:103BB0001DF015921596DEEF1DF01582C70E08EC6C
:103BC0000CF0E8CF00F10101008115A20091C70EB1
:103BD0000C6E00C10BF0F1EC0BF0C70E08EC0CF012
:103BE000E8CF00F1010100B1F9EF1DF01592FAEFF5
:103BF0001DF0158204014C0E826F70EC0FF0040171
:103C0000640E826F70EC0FF004012C0E826F70EC6A
:103C10000FF015B213EF1EF00401300E826F70EC3E
:103C20000FF018EF1EF00401310E826F70EC0FF0F0
:103C30001EEF33F04BEC3BF084C333F158EC3BF018
:103C4000CFEC3AF0200E0C6E00C10BF0F1EC0BF053
:103C500000C12FF505012F51000A06E005012F5183
:103C6000010A02E025EC3EF004014C0E826F70EC7C
:103C70000FF004014D0E826F70EC0FF004012C0E5A
:103C8000826F70EC0FF00AEC3BF02FC500F193EC63
:103C90003AF033C182F40401300E822770EC0FF049
:103CA000D4EF27F003EF46F004014C0E826F70EC66
:103CB0000FF00401630E826F70EC0FF0E3EC3CF048
:103CC00004012C0E826F70EC0FF069EC1EF0D4EF43
:103CD00027F00AEC3BF0B5C500F10101003B0F0EE7
:103CE000001793EC3AF033C182F40401300E8227BE
:103CF00070EC0FF0B5C500F101010F0E01010017C6
:103D000093EC3AF033C182F40401300E822770EC58
:103D10000FF004012D0E826F70EC0FF0B4C500F1AE
:103D20000101003B0F0E001793EC3AF033C182F40F
:103D30000401300E822770EC0FF0B4C500F10101D0
:103D40000F0E0101001793EC3AF033C182F4040125
:103D5000300E822770EC0FF004012D0E826F70EC94
:103D60000FF0B3C500F10101003B0F0E001793ECFB
:103D70003AF033C182F40401300E822770EC0FF068
:103D8000B3C500F101010F0E0101001793EC3AF0E9
:103D900033C182F40401300E822770EC0FF004016D
:103DA000200E826F70EC0FF0B2C500F10F0E010112
:103DB000001793EC3AF033C182F40401300E8227ED
:103DC00070EC0FF00401200E826F70EC0FF0B1C5A3
:103DD00000F101010101003B0F0E001793EC3AF0D6
:103DE00033C182F40401300E822770EC0FF0B1C5AC
:103DF00000F101010F0E0101001793EC3AF033C1FD
:103E000082F40401300E822770EC0FF004013A0EA8
:103E1000826F70EC0FF0B0C500F10101003B0F0E96
:103E2000001793EC3AF033C182F40401300E82277C
:103E300070EC0FF0B0C500F101010F0E0101001789
:103E400093EC3AF033C182F40401300E822770EC17
:103E50000FF004013A0E826F70EC0FF0AFC500F165
:103E60000101003B0F0E001793EC3AF033C182F4CE
:103E70000401300E822770EC0FF0AFC500F1010194
:103E80000F0E001793EC3AF033C182F40401300EA8
:103E9000822770EC0FF0120084C3E8FF0F0BE83AA2
:103EA000E8CFB5F585C3E8FF0F0B0501B51387C350
:103EB000E8FF0F0BE83AE8CFB4F588C3E8FF0F0B33
:103EC0000501B4138AC3E8FF0F0BE83AE8CFB3F556
:103ED0008BC3E8FF0F0B0501B3138DC3E8FF0F0B76
:103EE000E8CFB2F58FC3E8FF0F0BE83AE8CFB1F5A2
:103EF00090C3E8FF0F0B0501B11392C3E8FF0F0B4E
:103F0000E83AE8CFB0F593C3E8FF0F0B0501B01313
:103F100095C3E8FF0F0BE83AE8CFAFF596C3E8FF8B
:103F20000F0B0501AF133EEC3DF004014C0E826F08
:103F300070EC0FF00401430E826F70EC0FF05EEF37
:103F40001EF0078404014C0E826F70EC0FF0040128
:103F5000370E826F70EC0FF004012C0E826F70EC44
:103F60000FF005012E51130A06E005012E51170A24
:103F70000DE03CEF20F00101000E006F000E016F1C
:103F8000100E026F000E036FCFEF1FF00101000E45
:103F9000006F000E016F000E026F010E036F93ECB5
:103FA0003AF02AC182F40401300E822770EC0FF03F
:103FB0002BC182F40401300E822770EC0FF02CC16B
:103FC00082F40401300E822770EC0FF02DC182F4D0
:103FD0000401300E822770EC0FF02EC182F4040130
:103FE000300E822770EC0FF02FC182F40401300EE6
:103FF000822770EC0FF030C182F40401300E82276A
:1040000070EC0FF031C182F40401300E822770ECA5
:104010000FF032C182F40401300E822770EC0FF0F1
:1040200033C182F40401300E822770EC0FF00401DA
:104030002C0E826F70EC0FF00101200E006F000E4D
:10404000016F000E026F000E036F93EC3AF031C166
:1040500082F40401300E822770EC0FF032C182F43A
:104060000401300E822770EC0FF033C182F404019A
:10407000300E822770EC0FF00794D4EF27F0050183
:10408000216B226B236B246B04014C0E826F70EC4E
:104090000FF00401380E826F70EC0FF004012C0E4B
:1040A000826F70EC0FF00101200E006F000E016FA7
:1040B000000E026F000E036F93EC3AF02AC182F4F7
:1040C0000401300E822770EC0FF02BC182F4040142
:1040D000300E822770EC0FF02CC182F40401300EF8
:1040E000822770EC0FF02DC182F40401300E82277C
:1040F00070EC0FF02EC182F40401300E822770ECB8
:104100000FF02FC182F40401300E822770EC0FF003
:1041100030C182F40401300E822770EC0FF031C1FF
:1041200082F40401300E822770EC0FF032C182F469
:104130000401300E822770EC0FF033C182F40401C9
:10414000300E822770EC0FF004012C0E826F70ECA1
:104150000FF025C500F126C501F127C502F128C5DC
:1041600003F10101200E046F000E056F000E066FB3
:10417000000E076F26EC3AF000C133F501C134F5AB
:1041800002C135F503C136F593EC3AF02AC182F449
:104190000401300E822770EC0FF02BC182F4040171
:1041A000300E822770EC0FF02CC182F40401300E27
:1041B000822770EC0FF02DC182F40401300E8227AB
:1041C00070EC0FF02EC182F40401300E822770ECE7
:1041D0000FF02FC182F40401300E822770EC0FF033
:1041E00030C182F40401300E822770EC0FF031C12F
:1041F00082F40401300E822770EC0FF032C182F499
:104200000401300E822770EC0FF033C182F40401F8
:10421000300E822770EC0FF07AEC0FF00501336757
:1042200019EF21F0346719EF21F0356719EF21F00C
:10423000366702D0B8EF21F0129E129C21C500F122
:1042400022C501F123C502F124C503F1899A400E6C
:10425000C76E200EC66E9E96C69E0B0EC96EFF0ED2
:104260009EB602D0E82EFCD79E96C69E02C1C9FF1C
:10427000FF0E9EB602D0E82EFCD79E96C69E01C1C8
:10428000C9FFFF0E9EB602D0E82EFCD79E96C69EB2
:1042900000C1C9FFFF0E9EB602D0E82EFCD79E9645
:1042A000C69EC952FF0E9EB602D0E82EFCD705016D
:1042B000200E326F040114EE00F080517F0BE126D6
:1042C0009E96C69EC952FF0E9EB602D0E82EFCD71F
:1042D000C9CFE7FF0401802B0501322F5AEF21F0EF
:1042E000898A33C500F134C501F135C502F136C5FF
:1042F00003F10101010E046F000E056F000E066F41
:10430000000E076FF5EC39F000C133F501C134F54B
:1043100002C135F503C136F50501336797EF21F08A
:10432000346797EF21F0356797EF21F0366702D0B9
:10433000B8EF21F021C500F122C501F123C502F13A
:1043400024C503F10101200E046F000E056F000E5D
:10435000066F000E076FFAEC39F000C121F501C1BC
:1043600022F502C123F503C124F5128E20EF33F0AC
:104370000401450E826F70EC0FF004014F0E826F46
:1043800070EC0FF00401460E826F70EC0FF0D4EF6A
:1043900027F007845DEC45F00AEC3BF02DC500F1F9
:1043A00093EC3AF004014C0E826F70EC0FF00401B4
:1043B000300E826F70EC0FF004012C0E826F70ECE7
:1043C0000FF031C182F40401300E822770EC0FF03F
:1043D00032C182F40401300E822770EC0FF033C139
:1043E00082F40401300E822770EC0FF004012C0ED1
:1043F000826F70EC0FF00AEC3BF02EC500F193ECED
:104400003AF031C182F40401300E822770EC0FF0D3
:1044100032C182F40401300E822770EC0FF033C1F8
:1044200082F40401300E822770EC0FF00794D4EF71
:1044300027F004014C0E826F70EC0FF00401650E42
:10444000826F70EC0FF001EC3FF0D4EF27F0040125
:104450004C0E826F70EC0FF00401450E826F70EC11
:104460000FF018EC3FF0D4EF27F004014C0E826FF0
:1044700070EC0FF00401620E826F70EC0FF046ECEE
:104480003FF0D4EF27F004014C0E826F70EC0FF078
:104490000401420E826F70EC0FF02FEC3FF0D4EF6E
:1044A00027F004014C0E826F70EC0FF00401760EC1
:1044B000826F70EC0FF004012C0E826F70EC0FF025
:1044C00010A807D00401310E826F70EC0FF0D4EF0A
:1044D00027F00401300E826F70EC0FF0D4EF27F05C
:1044E00004014C0E826F70EC0FF004015A0E826FC3
:1044F00070EC0FF004012C0E826F70EC0FF05DEC8D
:1045000045F00AEC3BF005012E51130A06E00501C7
:104510002E51170A0DE0A1EF22F00101000E006FED
:10452000000E016F100E026F000E036FA1EF22F05C
:104530000101000E006F000E016F000E026F010EF0
:10454000036F0101200E046F000E056F000E066F51
:10455000000E076F26EC3AF093EC3AF02AC182F491
:104560000401300E822770EC0FF02BC182F404019D
:10457000300E822770EC0FF02CC182F40401300E53
:10458000822770EC0FF02DC182F40401300E8227D7
:1045900070EC0FF02EC182F40401300E822770EC13
:1045A0000FF02FC182F40401300E822770EC0FF05F
:1045B00030C182F40401300E822770EC0FF031C15B
:1045C00082F40401300E822770EC0FF032C182F4C5
:1045D0000401300E822770EC0FF033C182F4040125
:1045E000300E822770EC0FF0D4EF27F0078404011F
:1045F0004C0E826F70EC0FF00401310E826F70EC84
:104600000FF004012C0E826F70EC0FF025C500F145
:1046100026C501F127C502F128C503F10101200ECD
:10462000046F000E056F000E066F000E076F26EC7C
:104630003AF093EC3AF02AC182F40401300E82275A
:1046400070EC0FF02BC182F40401300E822770EC65
:104650000FF02CC182F40401300E822770EC0FF0B1
:104660002DC182F40401300E822770EC0FF02EC1B0
:1046700082F40401300E822770EC0FF02FC182F417
:104680000401300E822770EC0FF030C182F4040177
:10469000300E822770EC0FF031C182F40401300E2D
:1046A000822770EC0FF032C182F40401300E8227B1
:1046B00070EC0FF033C182F40401300E822770ECED
:1046C0000FF00794D4EF27F0078404014C0E826F9B
:1046D00070EC0FF00401320E826F70EC0FF035ECCD
:1046E00041F00794D4EF27F0078437B07AEF23F036
:1046F0008DEF23F0010E166E04014C0E826F70ECEC
:104700000FF00401330E826F70EC0FF092EC41F069
:10471000000E166E079401EF23F0020E166E92EC57
:1047200041F08B800501010E306F3C0E316F0101AD
:104730005E6B5F6B606B616B626B636B646B656B15
:10474000666B676B686B696B536B546BCF6ACE6A31
:104750000F9A0F9C0F9E030E166E04014C0E826F73
:1047600070EC0FF00401330E826F70EC0FF0040157
:104770002C0E826F70EC0FF004012D0E826F70EC26
:104780000FF00401310E826F70EC0FF01EEF33F06A
:1047900092EC41F0000E166E8B9020EF33F0078400
:1047A00004014C0E826F70EC0FF00401340E826F26
:1047B00070EC0FF004012C0E826F70EC0FF04BECDC
:1047C0003BF084C32AF185C32BF186C32CF187C348
:1047D0002DF188C32EF189C32FF18AC330F18BC329
:1047E00031F18CC332F18DC333F10101296B58ECE7
:1047F0003BF0CFEC3AF0200E046F000E056F000E78
:10480000066F000E076F06EC3AF000C121F501C1FA
:1048100022F502C123F503C124F510EC45F038C59B
:10482000AFF539C5B0F53AC5B1F53BC5B2F53CC5F4
:10483000B3F53DC5B4F53EC5B5F569EC1EF0040110
:104840002C0E826F70EC0FF03FC500F140C501F1F6
:1048500041C502F142C503F10101000E046F000ED3
:10486000056F010E066F000E076F26EC3AF093EC11
:104870003AF029673EEF24F043EF24F004012D0EB7
:10488000826F70EC0FF030C182F40401300E822789
:1048900070EC0FF031C182F40401300E822770EC0D
:1048A0000FF004012E0E826F70EC0FF032C182F413
:1048B0000401300E822770EC0FF033C182F4040142
:1048C000300E822770EC0FF004012C0E826F70EC1A
:1048D0000FF00AEC3BF043C500F144C501F14AEC8E
:1048E00034F004012C0E826F70EC0FF00AEC3BF0F8
:1048F00045C500F193EC3AF031C182F40401300E69
:10490000822770EC0FF032C182F40401300E82274E
:1049100070EC0FF033C182F40401300E822770EC8A
:104920000FF004012C0E826F70EC0FF00101036B8D
:10493000026B4CC501F14BC500F101AFA5EF24F0AE
:104940000101FF0E026FFF0E036F93EC3AF029672F
:10495000ACEF24F0B1EF24F004012D0E826F70EC67
:104960000FF02FC182F40401300E822770EC0FF09B
:1049700030C182F40401300E822770EC0FF031C197
:1049800082F40401300E822770EC0FF032C182F401
:104990000401300E822770EC0FF033C182F4040161
:1049A000300E822770EC0FF004012C0E826F70EC39
:1049B0000FF00101036B026B4EC501F14DC500F113
:1049C00001AFE8EF24F00101FF0E026FFF0E036F4D
:1049D00093EC3AF02967EFEF24F0F4EF24F00401B0
:1049E0002D0E826F70EC0FF02FC182F40401300E97
:1049F000822770EC0FF030C182F40401300E822760
:104A000070EC0FF031C182F40401300E822770EC9B
:104A10000FF032C182F40401300E822770EC0FF0E7
:104A200033C182F40401300E822770EC0FF00401D0
:104A30002C0E826F70EC0FF00101036B026B50C5FE
:104A400001F14FC500F101AF2BEF25F00101FF0E81
:104A5000026FFF0E036F93EC3AF0296732EF25F0F7
:104A600037EF25F004012D0E826F70EC0FF02FC18F
:104A700082F40401300E822770EC0FF030C182F412
:104A80000401300E822770EC0FF031C182F4040172
:104A9000300E822770EC0FF032C182F40401300E28
:104AA000822770EC0FF033C182F40401300E8227AC
:104AB00070EC0FF004012C0E826F70EC0FF001010E
:104AC000036B026B52C501F151C500F101AF6EEFEE
:104AD00025F00101FF0E026FFF0E036F93EC3AF019
:104AE000296775EF25F07AEF25F004012D0E826F0E
:104AF00070EC0FF02FC182F40401300E822770ECAD
:104B00000FF030C182F40401300E822770EC0FF0F8
:104B100031C182F40401300E822770EC0FF032C1F3
:104B200082F40401300E822770EC0FF033C182F45E
:104B30000401300E822770EC0FF004012C0E826FFE
:104B400070EC0FF00101036B026B54C501F153C50A
:104B500000F101AFB1EF25F00101FF0E026FFF0E72
:104B6000036F93EC3AF02967B8EF25F0BDEF25F01D
:104B700004012D0E826F70EC0FF02FC182F404013E
:104B8000300E822770EC0FF030C182F40401300E39
:104B9000822770EC0FF031C182F40401300E8227BD
:104BA00070EC0FF032C182F40401300E822770ECF9
:104BB0000FF033C182F40401300E822770EC0FF045
:104BC00004012C0E826F70EC0FF00101036B026B7D
:104BD00056C501F155C500F101AFF4EF25F0010113
:104BE000FF0E026FFF0E036F93EC3AF02967FBEFA5
:104BF00025F000EF26F004012D0E826F70EC0FF00F
:104C00002FC182F40401300E822770EC0FF030C106
:104C100082F40401300E822770EC0FF031C182F46F
:104C20000401300E822770EC0FF032C182F40401CF
:104C3000300E822770EC0FF033C182F40401300E85
:104C4000822770EC0FF004012C0E826F70EC0FF0D5
:104C50000101036B026B4AC501F149C500F101AFC7
:104C600037EF26F00101FF0E026FFF0E036F93EC8A
:104C70003AF029673EEF26F043EF26F004012D0EAF
:104C8000826F70EC0FF02FC182F40401300E822786
:104C900070EC0FF030C182F40401300E822770EC0A
:104CA0000FF031C182F40401300E822770EC0FF056
:104CB00032C182F40401300E822770EC0FF033C150
:104CC00082F40401300E822770EC0FF004012C0EE8
:104CD000826F70EC0FF037C5E8FFE8B806D004012A
:104CE000300E826F70EC0FF005D00401310E826F30
:104CF00070EC0FF00794D4EF27F04BEC3BF085C33A
:104D00002AF186C32BF187C32CF188C32DF189C307
:104D10002EF18AC32FF18BC330F18CC331F18DC3D7
:104D200032F18EC333F10101296B58EC3BF0CFEC2B
:104D30003AF00101010E046F000E056F000E066FC0
:104D4000000E076FF5EC39F0100E046F000E056FC2
:104D5000000E066F000E076F06EC3AF000C129F551
:104D600001C12AF502C12BF503C12CF5BCEC40F0C2
:104D700004014C0E826F70EC0FF00401460E826F3E
:104D800070EC0FF004012C0E826F70EC0FF025C553
:104D900000F126C501F127C502F128C503F1010183
:104DA000100E046F000E056F000E066F000E076FE9
:104DB00026EC3AF093EC3AF02AC182F40401300E6A
:104DC000822770EC0FF02BC182F40401300E822791
:104DD00070EC0FF02CC182F40401300E822770ECCD
:104DE0000FF02DC182F40401300E822770EC0FF019
:104DF0002EC182F40401300E822770EC0FF02FC117
:104E000082F40401300E822770EC0FF030C182F47E
:104E10000401300E822770EC0FF031C182F40401DE
:104E2000300E822770EC0FF032C182F40401300E94
:104E3000822770EC0FF033C182F40401300E822718
:104E400070EC0FF0D4EF27F037B029EF27F0020E07
:104E5000166E92EC41F000011650020AD8B447EFEA
:104E600027F005012F51010AD8B43DEF27F015B204
:104E700042EF27F081BA42EF27F0000E166E15843C
:104E800020EF33F0050E166E158403EF46F08B808D
:104E900001015E6B5F6B606B616B626B636B646B7C
:104EA000656B666B676B686B696B536B546BCF6A32
:104EB000CE6A0F9A0F9C0F9E030E166E20EF33F0F2
:104EC00092EC41F005012F51010AD8B46EEF27F0A2
:104ED00015B273EF27F081BA73EF27F0000E166E4C
:104EE000158420EF33F0050E166E158403EF46F09F
:104EF00004014C0E826F70EC0FF00401350E826FCE
:104F000070EC0FF004012C0E826F70EC0FF00AECC5
:104F10003BF00784B9C500F1079493EC3AF031C136
:104F200082F40401300E822770EC0FF032C182F45B
:104F30000401300E822770EC0FF033C182F40401BB
:104F4000300E822770EC0FF0D4EF27F055EC41F0D3
:104F50000AEC3BF037C500F193EC3AF004014C0E3B
:104F6000826F70EC0FF00401360E826F70EC0FF060
:104F700004012C0E826F70EC0FF031C182F4040139
:104F8000300E822770EC0FF032C182F40401300E33
:104F9000822770EC0FF033C182F40401300E8227B7
:104FA00070EC0FF0D4EF27F07AEC0FF020EF33F035
:104FB00004014C0E826F70EC0FF00401500E826FF2
:104FC00070EC0FF004012C0E826F70EC0FF085C3B3
:104FD0002AF186C32BF187C32CF188C32DF189C335
:104FE0002EF18AC32FF18BC330F18CC331F18DC305
:104FF00032F18EC333F1010158EC3BF0CFEC3AF0C3
:1050000003018451530A0DE0030184514D0A38E035
:105010000401780E826F70EC0FF07AEC0FF020EF45
:1050200033F00401530E826F70EC0FF0250E0C6EFE
:1050300000C10BF0F1EC0BF0260E0C6E01C10BF071
:10504000F1EC0BF0270E0C6E02C10BF0F1EC0BF043
:10505000280E0C6E03C10BF0F1EC0BF000C157F5FC
:1050600001C158F502C159F503C15AF500C15BF5FC
:1050700001C15CF502C15DF503C15EF5B5EF28F035
:1050800004014D0E826F70EC0FF0290E0C6E00C102
:105090000BF0F1EC0BF000C15FF500C160F5B5EF6E
:1050A00028F004014C0E826F70EC0FF00401540ED6
:1050B000826F70EC0FF004012C0E826F70EC0FF019
:1050C00084C32AF185C32BF186C32CF187C32DF14C
:1050D00088C32EF189C32FF18AC330F18BC331F11C
:1050E0008DC332F18EC333F1010158EC3BF0CFECAC
:1050F0003AF00101000E046F000E056F010E066FFD
:10510000000E076F06EC3AF0210E0C6E00C10BF09A
:10511000F1EC0BF0220E0C6E01C10BF0F1EC0BF078
:10512000230E0C6E02C10BF0F1EC0BF0240E0C6E92
:1051300003C10BF0F1EC0BF000C161F501C162F5A8
:1051400002C163F503C164F5B5EF28F004014C0E0C
:10515000826F70EC0FF00401490E826F70EC0FF05B
:1051600004012C0E826F70EC0FF0250E08EC0CF091
:10517000E8CF00F1260E08EC0CF0E8CF01F1270E85
:1051800008EC0CF0E8CF02F1280E08EC0CF0E8CFA8
:1051900003F193EC3AF056EC38F00401730E826F91
:1051A00070EC0FF004012C0E826F70EC0FF00AEC23
:1051B0003BF0290E08EC0CF0E8CF00F193EC3AF04C
:1051C00056EC38F004016D0E826F70EC0FF00401A4
:1051D0002C0E826F70EC0FF05BC500F15CC501F125
:1051E0005DC502F15EC503F193EC3AF056EC38F080
:1051F0000401730E826F70EC0FF004012C0E826FAD
:1052000070EC0FF00AEC3BF060C500F193EC3AF063
:1052100056EC38F004016D0E826F70EC0FF0040153
:105220002C0E826F70EC0FF061C500F162C501F1C8
:1052300063C502F164C503F13BEC33F004012C0EAD
:10524000826F70EC0FF07AEC0FF020EF33F083C335
:105250002AF184C32BF185C32CF186C32DF187C3BA
:105260002EF188C32FF189C330F18AC331F18BC38A
:1052700032F18CC333F1010158EC3BF0CFEC3AF042
:10528000160E0C6E00C10BF0F1EC0BF0170E0C6E4D
:1052900001C10BF0F1EC0BF0180E0C6E02C10BF01B
:1052A000F1EC0BF0190E0C6E03C10BF0F1EC0BF0EE
:1052B00000C18EF101C18FF102C190F103C191F1E2
:1052C00000C192F101C193F102C194F103C195F1C2
:1052D00009EF2AF083C32AF184C32BF185C32CF193
:1052E00086C32DF187C32EF188C32FF189C330F116
:1052F0008AC331F18BC332F18CC333F1010158EC15
:105300003BF0CFEC3AF000C18EF101C18FF102C148
:1053100090F103C191F100C192F101C193F102C179
:1053200094F103C195F109EF2AF083C32AF184C3F4
:105330002BF185C32CF186C32DF187C32EF188C3D1
:105340002FF189C330F18AC331F18CC332F18DC39F
:1053500033F1010158EC3BF0CFEC3AF00101000EC3
:10536000046F000E056F010E066F000E076F06EC4E
:105370003AF01A0E0C6E00C10BF0F1EC0BF01B0EA4
:105380000C6E01C10BF0F1EC0BF01C0E0C6E02C1A7
:105390000BF0F1EC0BF01D0E0C6E03C10BF0F1ECF9
:1053A0000BF000C196F101C197F102C198F103C160
:1053B00099F109EF2AF083C32AF184C32BF185C345
:1053C0002CF186C32DF187C32EF188C32FF189C339
:1053D00030F18AC331F18CC332F18DC333F1010155
:1053E00058EC3BF0CFEC3AF00101000E046F000ED8
:1053F000056F010E066F000E076F06EC3AF000C154
:1054000096F101C197F102C198F103C199F109EF39
:105410002AF0160E08EC0CF0E8CF00F1170E08EC9D
:105420000CF0E8CF01F1180E08EC0CF0E8CF02F117
:10543000190E08EC0CF0E8CF03F193EC3AF056ECBF
:1054400038F00401730E826F70EC0FF004012C0E23
:10545000826F70EC0FF08EC100F18FC101F190C12D
:1054600002F191C103F193EC3AF056EC38F00401EB
:10547000730E826F70EC0FF004012C0E826F70ECD3
:105480000FF01A0E08EC0CF0E8CF00F11B0E08EC40
:105490000CF0E8CF01F11C0E08EC0CF0E8CF02F1A3
:1054A0001D0E08EC0CF0E8CF03F13BEC33F00401E7
:1054B0002C0E826F70EC0FF096C100F197C101F1D4
:1054C00098C102F199C103F13BEC33F07AEC0FF093
:1054D00020EF33F00401690E826F70EC0FF00401CD
:1054E0002C0E826F70EC0FF00101040E006F000EA5
:1054F000016F000E026F000E036F93EC3AF02CC1A7
:1055000082F40401300E822770EC0FF02DC182F47A
:105510000401300E822770EC0FF02EC182F40401DA
:10552000300E822770EC0FF02FC182F40401300E90
:10553000822770EC0FF030C182F40401300E822714
:1055400070EC0FF031C182F40401300E822770EC50
:105550000FF032C182F40401300E822770EC0FF09C
:1055600033C182F40401300E822770EC0FF0040185
:105570002C0E826F70EC0FF001010B0E006F000E0D
:10558000016F000E026F000E036F93EC3AF02CC116
:1055900082F40401300E822770EC0FF02DC182F4EA
:1055A0000401300E822770EC0FF02EC182F404014A
:1055B000300E822770EC0FF02FC182F40401300E00
:1055C000822770EC0FF030C182F40401300E822784
:1055D00070EC0FF031C182F40401300E822770ECC0
:1055E0000FF032C182F40401300E822770EC0FF00C
:1055F00033C182F40401300E822770EC0FF00401F5
:105600002C0E826F70EC0FF001014A0E006F000E3D
:10561000016F000E026F000E036F93EC3AF02CC185
:1056200082F40401300E822770EC0FF02DC182F459
:105630000401300E822770EC0FF02EC182F40401B9
:10564000300E822770EC0FF02FC182F40401300E6F
:10565000822770EC0FF030C182F40401300E8227F3
:1056600070EC0FF031C182F40401300E822770EC2F
:105670000FF032C182F40401300E822770EC0FF07B
:1056800033C182F40401300E822770EC0FF0040164
:105690002C0E826F70EC0FF0200EF86EF76AF66A2F
:1056A00004010900F5CF82F470EC0FF00900F5CF8A
:1056B00082F470EC0FF00900F5CF82F470EC0FF07B
:1056C0000900F5CF82F470EC0FF00900F5CF82F4F9
:1056D00070EC0FF00900F5CF82F470EC0FF00900C8
:1056E000F5CF82F470EC0FF00900F5CF82F470EC86
:1056F0000FF07AEC0FF020EF33F08351630AD8A457
:105700001EEF33F08451610AD8A41EEF33F08551A7
:105710006C0AD8A41EEF33F08651410A3FE086514F
:10572000440A1BE08651420AD8B4E1EF2BF08651BF
:10573000350AD8B4AAEF34F08651360AD8B4FFEF50
:1057400034F08651370AD8B468EF35F08651380AFC
:10575000D8B4C6EF35F01EEF33F00798079A04016E
:105760007A0E826F70EC0FF00401780E826F70EC8D
:105770000FF00401640E826F70EC0FF00401550EFF
:10578000826F70EC0FF0CAEF2BF004014C0E826FA9
:1057900070EC0FF07AEC0FF020EF33F00788079AE7
:1057A00004017A0E826F70EC0FF00401410E826FDB
:1057B00070EC0FF00401610E826F70EC0FF0BEEF21
:1057C0002BF00798078A04017A0E826F70EC0FF0B5
:1057D0000401420E826F70EC0FF00401610E826FC3
:1057E00070EC0FF0BEEF2BF001016667FFEF2BF0BE
:1057F0006767FFEF2BF06867FFEF2BF0696716D044
:1058000001014F670BEF2CF050670BEF2CF0516745
:105810000BEF2CF052670AD00101000E006F000E52
:10582000016F000E026F000E036F120011B80AD054
:105830000101620E046F010E056F000E066F000E6F
:10584000076F09D00101A70E046F020E056F000E4D
:10585000066F000E076F66C100F167C101F168C1F4
:1058600002F169C103F1F5EC39F003BFA8EF2CF0A8
:10587000119A119C0101000E046FA80E056F550EC0
:10588000066F020E076F66C100F167C101F168C1C2
:1058900002F169C103F166C18AF167C18BF168C188
:1058A0008CF169C18DF1F5EC39F003BF0BD001012A
:1058B000000E8A6FA80E8B6F550E8C6F020E8D6FC7
:1058C000118A119C0E0E08EC0CF0E8CF18F10F0EA7
:1058D00008EC0CF0E8CF19F1100E08EC0CF0E8CF52
:1058E0001AF1110E08EC0CF0E8CF1BF13EEC39F088
:1058F0008AC104F18BC105F18CC106F18DC107F19C
:10590000F5EC39F0078202EC39F03EEC39F0079201
:1059100002EC39F08AC100F18BC101F18CC102F1B6
:105920008DC103F1079202EC39F0CC0E046FE00E4A
:10593000056F870E066F050E076FF5EC39F000C195
:1059400018F101C119F102C11AF103C11BF140D0D4
:1059500013AAADEF2CF0138E139A119C119A01012A
:10596000800E006F1A0E016F060E026F000E036F9D
:105970004FC104F150C105F151C106F152C107F107
:10598000F5EC39F003AF05D00AEC3BF0118C119A1D
:1059900012000E0E08EC0CF0E8CF18F10F0E08EC18
:1059A0000CF0E8CF19F1100E08EC0CF0E8CF1AF16A
:1059B000110E08EC0CF0E8CF1BF14FC100F150C103
:1059C00001F151C102F152C103F1078202EC39F039
:1059D00018C100F119C101F11AC102F11BC103F193
:1059E00012000784BAC166F1BBC167F1BCC168F19E
:1059F000BDC169F14BC14FF14CC150F14DC151F1E5
:105A00004EC152F157C159F158C15AF107940101E1
:105A1000666712EF2DF0676712EF2DF0686712EFDF
:105A20002DF0696716D001014F671EEF2DF050670A
:105A30001EEF2DF051671EEF2DF052670AD00101C5
:105A4000000E006F000E016F000E026F000E036F5C
:105A5000120011B80AD00101620E046F010E056F29
:105A6000000E066F000E076F09D00101A70E046F2C
:105A7000020E056F000E066F000E076F66C100F183
:105A800067C101F168C102F169C103F1F5EC39F0B8
:105A900003BFAAEF2DF00101000E046FA80E056FE1
:105AA000550E066F020E076F66C100F167C101F166
:105AB00068C102F169C103F166C18AF167C18BF166
:105AC00068C18CF169C18DF1F5EC39F003BF09D0E3
:105AD0000101000E8A6FA80E8B6F550E8C6F020E9F
:105AE0008D6F3EEC39F000C104F101C105F102C136
:105AF00006F103C107F1000E006FA00E016F980EB2
:105B0000026F7B0E036F26EC3AF000C118F101C161
:105B100019F102C11AF103C11BF1000E006FA00EB2
:105B2000016F980E026F7B0E036F8AC104F18BC167
:105B300005F18CC106F18DC107F126EC3AF018C1D0
:105B400004F119C105F11AC106F11BC107F1F5EC09
:105B500039F012000101A80E006F610E016F000EF6
:105B6000026F000E036F4FC104F150C105F151C126
:105B700006F152C107F1F5EC39F003AF0AD001018B
:105B8000A80E006F610E016F000E026F000E036F12
:105B900000D0C80E006FAF0E016F000E026F000E36
:105BA000036F4FC104F150C105F151C106F152C15B
:105BB00007F106EC3AF012000401730E826F70ECEC
:105BC0000FF004012C0E826F70EC0FF0078462C19D
:105BD00066F163C167F164C168F165C169F14BC1E8
:105BE0004FF14CC150F14DC151F14EC152F157C16D
:105BF00059F158C15AF1079402EC2EF07AEC0FF0EB
:105C000020EF33F066C100F167C101F168C102F114
:105C100069C103F1010193EC3AF056EC38F004014C
:105C2000630E826F70EC0FF004012C0E826F70EC2B
:105C30000FF04FC100F150C101F151C102F152C149
:105C400003F1010193EC3AF056EC38F00401660ED2
:105C5000826F70EC0FF004012C0E826F70EC0FF06D
:105C60000AEC3BF059C100F15AC101F1010193EC7A
:105C70003AF056EC38F00401740E826F70EC0FF0BD
:105C8000120010820401530E826F70EC0FF00401B9
:105C90002C0E826F70EC0FF083C32AF184C32BF1BA
:105CA00085C32CF186C32DF187C32EF188C32FF154
:105CB00089C330F18AC331F18BC332F18CC333F124
:105CC000010158EC3BF0CFEC3AF000C166F101C1A4
:105CD00067F102C168F103C169F18EC32AF18FC374
:105CE0002BF190C32CF191C32DF192C32EF193C3EC
:105CF0002FF194C330F195C331F196C332F197C3BC
:105D000033F1010158EC3BF0CFEC3AF000C14FF118
:105D100001C150F102C151F103C152F14BEC3BF012
:105D200099C32FF19AC330F19BC331F19CC332F177
:105D30009DC333F1010158EC3BF0CFEC3AF000C1C8
:105D400059F101C15AF102EC2EF004012C0E826FC0
:105D500070EC0FF0BCEF2EF0118E1CA002D01CAE28
:105D6000108C1BBE02D01BA4108E03018251520A5C
:105D700002E10F8201D00F928251750A02E1108474
:105D800001D010948251550A02E1108601D010967C
:105D90008351310A03E11382138402D013921394C6
:105DA00003018351660A01E056D00401660E826F3A
:105DB00070EC0FF004012C0E826F70EC0FF0F1EC20
:105DC0002CF093EC3AF02AC182F40401300E8227C1
:105DD00070EC0FF02BC182F40401300E822770ECBE
:105DE0000FF02CC182F40401300E822770EC0FF00A
:105DF0002DC182F40401300E822770EC0FF02EC109
:105E000082F40401300E822770EC0FF02FC182F46F
:105E10000401300E822770EC0FF030C182F40401CF
:105E2000300E822770EC0FF031C182F40401300E85
:105E3000822770EC0FF032C182F40401300E822709
:105E400070EC0FF033C182F40401300E822770EC45
:105E50000FF01EEF33F011A003D011A401D0108475
:105E6000078410B295EF2FF010A479EF2FF0BAC18C
:105E700066F1BBC167F1BCC168F1BDC169F1BEC1CA
:105E80006AF1BFC16BF1C0C16CF1C1C16DF1C2C19A
:105E90006EF1C3C16FF1C4C170F1C5C171F1C6C16A
:105EA00072F1C7C173F1C8C174F1C9C175F1CAC13A
:105EB00076F1CBC177F1CCC178F1CDC179F1CEC10A
:105EC0007AF1CFC17BF1D0C17CF1D1C17DF1D2C1DA
:105ED0007EF1D3C17FF1D4C180F1D5C181F1D6C1AA
:105EE00082F1D7C183F1D8C184F1D9C185F181EFA5
:105EF0002FF062C166F163C167F164C168F165C1E9
:105F000069F1BAC186F1BBC187F1BCC188F1BDC1DD
:105F100089F14BC14FF14CC150F14DC151F14EC10E
:105F200052F157C159F158C15AF107940FA0B7EF78
:105F30002FF001019667A4EF2FF09767A4EF2FF0E1
:105F40009867A4EF2FF09967A8EF2FF0B7EF2FF025
:105F5000F4EC2BF096C104F197C105F198C106F15C
:105F600099C107F1F5EC39F003BFE4EF32F0F4EC3E
:105F70002BF00101000E046F000E056F010E066F7D
:105F8000000E076F26EC3AF011A02AD011A228D0FB
:105F900093EC3AF0296701D005D004012D0E826FF1
:105FA00070EC0FF030C182F40401300E822770ECE7
:105FB0000FF031C182F40401300E822770EC0FF033
:105FC00032C182F40401300E822770EC0FF033C12D
:105FD00082F40401300E822770EC0FF07AEC0FF09F
:105FE00012A8C5D012981DC01EF01E3A1E42070E00
:105FF0001E1600011E50000AD8B483EF30F00001D5
:106000001E50010AD8B40FEF30F000011E50020AF2
:10601000D8B40DEF30F0B5EF30F0B5EF30F00AEC5A
:106020003BF02DC001F12EC000F1D89001330033B8
:10603000D890013300330101630E046F000E056F29
:10604000000E066F000E076F26EC3AF0280E046F64
:10605000000E056F000E066F000E076FF5EC39F0AD
:1060600000C130F00AEC3BF02BC001F1019F019D13
:106070002CC000F10101A40E046F000E056F000E8C
:10608000066F000E076F26EC3AF000C12FF000C13A
:1060900004F101C105F102C106F103C107F1640E6B
:1060A000006F000E016F000E026F000E036FF5EC23
:1060B00039F0050E046F000E056F000E066F000E1E
:1060C000076F26EC3AF000C104F101C105F102C1ED
:1060D00006F103C107F10AEC3BF030C000F1F5EC2A
:1060E00039F000C131F031C0E8FF050F305C03E743
:1060F0008A84B5EF30F031C0E8FF0A0F305C01E66A
:106100008A94B5EF30F000C124F101C125F102C13C
:1061100026F103C127F10AEC3BF010EC3BF01D50D7
:106120001F0BE8CF00F10101640E046F000E056F34
:10613000000E066F000E076F06EC3AF024C104F162
:1061400025C105F126C106F127C107F1F5EC39F0AB
:1061500003BF02D08A9401D08A8424C100F125C1F2
:1061600001F126C102F127C103F120EF33F000C194
:1061700024F101C125F102C126F103C127F110AEBE
:106180004DD0109E00C108F101C109F102C10AF110
:1061900003C10BF193EC3AF030C1E2F131C1E3F10C
:1061A00032C1E4F133C1E5F108C100F109C101F1E7
:1061B0000AC102F10BC103F101016C0E046F070E5D
:1061C000056F000E066F000E076FF5EC39F003BF88
:1061D00004D00101550EE66F1CD008C100F109C1C1
:1061E00001F10AC102F10BC103F10101A40E046F18
:1061F000060E056F000E066F000E076FF5EC39F006
:1062000003BF04D001017F0EE66F03D00101FF0E32
:10621000E66F1F8E11AEE4EF32F0119E24C100F143
:1062200025C101F126C102F127C103F111A005D05A
:1062300011A203D00FB0E4EF32F010A427EF31F039
:106240000401750E826F70EC0FF02CEF31F0040139
:10625000720E826F70EC0FF004012C0E826F70ECE6
:106260000FF093EC3AF029673BEF31F00401200E78
:10627000826F3EEF31F004012D0E826F70EC0FF053
:1062800030C182F40401300E822770EC0FF031C16E
:1062900082F40401300E822770EC0FF004012E0E00
:1062A000826F70EC0FF032C182F40401300E82274D
:1062B00070EC0FF033C182F40401300E822770ECD1
:1062C0000FF004016D0E826F70EC0FF004012C0EC4
:1062D000826F70EC0FF04FC100F150C101F151C15C
:1062E00002F152C103F1010193EC3AF056EC38F09F
:1062F0000401480E826F70EC0FF004017A0E826F79
:1063000070EC0FF004012C0E826F70EC0FF066C180
:1063100000F167C101F168C102F169C103F1010136
:1063200093EC3AF056EC38F00401630E826F70EC97
:106330000FF004012C0E826F70EC0FF066C100F1BB
:1063400067C101F168C102F169C103F101010A0EDF
:10635000046F000E056F000E066F000E076F06EC4F
:106360003AF0000E046F120E056F000E066F000E5D
:10637000076F26EC3AF093EC3AF02AC182F404015C
:10638000300E822770EC0FF02BC182F40401300E26
:10639000822770EC0FF02CC182F40401300E8227AA
:1063A00070EC0FF02DC182F40401300E822770ECE6
:1063B0000FF02EC182F40401300E822770EC0FF032
:1063C0002FC182F40401300E822770EC0FF030C12F
:1063D00082F40401300E822770EC0FF004012E0EBF
:1063E000826F70EC0FF031C182F40401300E82270D
:1063F00070EC0FF032C182F40401300E822770EC91
:106400000FF033C182F40401300E822770EC0FF0DC
:106410000401730E826F70EC0FF004012C0E826F7A
:1064200070EC0FF00AEC3BF059C100F15AC101F1D8
:106430004AEC34F013A26CEF32F004012C0E826FA0
:1064400070EC0FF086C166F187C167F188C168F111
:1064500089C169F1F4EC2BF00101000E046F000E0C
:10646000056F010E066F000E076F26EC3AF093ECF5
:106470003AF0296741EF32F00401200E826F44EFB9
:1064800032F004012D0E826F70EC0FF030C182F4F7
:106490000401300E822770EC0FF031C182F4040148
:1064A000300E822770EC0FF004012E0E826F70EC1C
:1064B0000FF032C182F40401300E822770EC0FF02D
:1064C00033C182F40401300E822770EC0FF0040116
:1064D0006D0E826F70EC0FF013A493EF32F0040195
:1064E0002C0E826F70EC0FF013AC81EF32F00401D0
:1064F000500E826F70EC0FF0139C1398139A93EF69
:1065000032F013AE8EEF32F00401460E826F70EC63
:106510000FF0139E1398139A93EF32F00401530E69
:10652000826F70EC0FF037B0AAEF32F004012C0E3E
:10653000826F70EC0FF08BB0A5EF32F00401440EC7
:10654000826F70EC0FF0AAEF32F00401530E826FED
:1065500070EC0FF00FB2B0EF32F00FA0E2EF32F0BC
:1065600004012C0E826F70EC0FF0200EF86EF76AAB
:10657000F66A04010900F5CF82F470EC0FF009000F
:10658000F5CF82F470EC0FF00900F5CF82F470ECD7
:106590000FF00900F5CF82F470EC0FF00900F5CF91
:1065A00082F470EC0FF00900F5CF82F470EC0FF07C
:1065B0000900F5CF82F470EC0FF00900F5CF82F4FA
:1065C00070EC0FF07AEC0FF00F90109E129820EF05
:1065D00033F00401630E826F70EC0FF004012C0E97
:1065E000826F70EC0FF026EC33F004012C0E826FFA
:1065F00070EC0FF099EC33F004012C0E826F70EC0C
:106600000FF015EC34F004012C0E826F70EC0FF0DB
:106610000101F80E006FCD0E016F660E026F030EC2
:10662000036F3BEC33F004012C0E826F70EC0FF023
:106630002BEC34F07AEC0FF020EF33F07AEC0FF023
:106640000301C26B079010922FEF36F0D8900E0E18
:1066500008EC0CF0E8CF00F10F0E08EC0CF0E8CFDE
:1066600001F1100E08EC0CF0E8CF02F1110E08EC6D
:106670000CF0E8CF03F10101000E046F000E056F6E
:10668000010E066F000E076F26EC3AF093EC3AF01D
:106690002AC182F40401300E822770EC0FF02BC166
:1066A00082F40401300E822770EC0FF02CC182F4CA
:1066B0000401300E822770EC0FF02DC182F404012A
:1066C000300E822770EC0FF02EC182F40401300EE0
:1066D000822770EC0FF02FC182F40401300E822764
:1066E00070EC0FF030C182F40401300E822770ECA0
:1066F0000FF031C182F40401300E822770EC0FF0EC
:1067000004012E0E826F70EC0FF032C182F404018E
:10671000300E822770EC0FF033C182F40401300E8A
:10672000822770EC0FF004016D0E826F70EC0FF099
:106730001200120E08EC0CF0E8CF00F1130E08EC7A
:106740000CF0E8CF01F1140E08EC0CF0E8CF02F1E8
:10675000150E08EC0CF0E8CF03F101010A0E046FEE
:10676000000E056F000E066F000E076F06EC3AF084
:10677000000E046F120E056F000E066F000E076FFD
:1067800026EC3AF093EC3AF02AC182F40401300E80
:10679000822770EC0FF02BC182F40401300E8227A7
:1067A00070EC0FF02CC182F40401300E822770ECE3
:1067B0000FF02DC182F40401300E822770EC0FF02F
:1067C0002EC182F40401300E822770EC0FF02FC12D
:1067D00082F40401300E822770EC0FF030C182F495
:1067E0000401300E822770EC0FF004012E0E826F30
:1067F00070EC0FF031C182F40401300E822770EC8E
:106800000FF032C182F40401300E822770EC0FF0D9
:1068100033C182F40401300E822770EC0FF00401C2
:10682000730E826F70EC0FF012000A0E08EC0CF081
:10683000E8CF00F10B0E08EC0CF0E8CF01F10C0EE4
:1068400008EC0CF0E8CF02F10D0E08EC0CF0E8CFEC
:1068500003F14AEF34F0060E08EC0CF0E8CF00F13B
:10686000070E08EC0CF0E8CF01F1080E08EC0CF074
:10687000E8CF02F1090E08EC0CF0E8CF03F14AEF83
:1068800034F001010AEC3BF0078457C100F158C114
:1068900001F107940101E80E046F800E056F000EF0
:1068A000066F000E076F06EC3AF0000E046F040E40
:1068B000056F000E066F000E076F26EC3AF0880E8B
:1068C000046F130E056F000E066F000E076FF5ECD8
:1068D00039F00A0E046F000E056F000E066F000EF1
:1068E000076F26EC3AF093EC3AF0010129677EEF4E
:1068F00034F00401200E826F81EF34F004012D0E7C
:10690000826F70EC0FF030C182F40401300E8227E8
:1069100070EC0FF031C182F40401300E822770EC6C
:106920000FF032C182F40401300E822770EC0FF0B8
:1069300004012E0E826F70EC0FF033C182F404015B
:10694000300E822770EC0FF00401430E826F70EC62
:106950000FF0120087C32AF188C32BF189C32CF1F1
:106960008AC32DF18BC32EF18CC32FF18DC330F16F
:106970008EC331F190C332F191C333F10101296B20
:1069800058EC3BF0CFEC3AF00101000E046F000E22
:10699000056F010E066F000E076F06EC3AF00E0E43
:1069A0000C6E00C10BF0F1EC0BF00F0E0C6E01C180
:1069B0000BF0F1EC0BF0100E0C6E02C10BF0F1ECD1
:1069C0000BF0110E0C6E03C10BF0F1EC0BF0040197
:1069D0007A0E826F70EC0FF004012C0E826F70EC57
:1069E0000FF00401350E826F70EC0FF004012C0ED5
:1069F000826F70EC0FF026EC33F0CAEF2BF087C3F8
:106A00002AF188C32BF189C32CF18AC32DF18BC3E2
:106A10002EF18CC32FF18DC330F18EC331F190C3B1
:106A200032F191C333F10101296B58EC3BF0CFEC0B
:106A30003AF0880E046F130E056F000E066F000EFD
:106A4000076FFAEC39F0000E046F040E056F000EAC
:106A5000066F000E076F06EC3AF00101E80E046FB6
:106A6000800E056F000E066F000E076F26EC3AF0E1
:106A70000A0E0C6E00C10BF0F1EC0BF00B0E0C6E5D
:106A800001C10BF0F1EC0BF00C0E0C6E02C10BF01F
:106A9000F1EC0BF00D0E0C6E03C10BF0F1EC0BF0F2
:106AA00004017A0E826F70EC0FF004012C0E826FDD
:106AB00070EC0FF00401360E826F70EC0FF00401E1
:106AC0002C0E826F70EC0FF015EC34F0CAEF2BF047
:106AD00087C32AF188C32BF189C32CF18AC32DF116
:106AE0008BC32EF18CC32FF18DC330F18FC331F1E5
:106AF00090C332F191C333F1010158EC3BF0CFEC7C
:106B00003AF0000E046F120E056F000E066F000EB5
:106B1000076F06EC3AF001010A0E046F000E056FD4
:106B2000000E066F000E076F26EC3AF0120E0C6E88
:106B300000C10BF0F1EC0BF0130E0C6E01C10BF069
:106B4000F1EC0BF0140E0C6E02C10BF0F1EC0BF03B
:106B5000150E0C6E03C10BF0F1EC0BF004017A0E74
:106B6000826F70EC0FF004012C0E826F70EC0FF04E
:106B70000401370E826F70EC0FF004012C0E826F4F
:106B800070EC0FF099EC33F0CAEF2BF087C32AF1C9
:106B900088C32BF189C32CF18AC32DF18BC32EF14D
:106BA0008CC32FF18DC330F18EC331F190C332F11C
:106BB00091C333F10101296B58EC3BF0CFEC3AF073
:106BC000880E046F130E056F000E066F000E076F20
:106BD000FAEC39F0000E046F040E056F000E066F1C
:106BE000000E076F06EC3AF00101E80E046F800E0C
:106BF000056F000E066F000E076F26EC3AF0060ECA
:106C00000C6E00C10BF0F1EC0BF0070E0C6E01C125
:106C10000BF0F1EC0BF0080E0C6E02C10BF0F1EC76
:106C20000BF0090E0C6E03C10BF0F1EC0BF004013C
:106C30007A0E826F70EC0FF004012C0E826F70ECF4
:106C40000FF00401380E826F70EC0FF004012C0E6F
:106C5000826F70EC0FF02BEC34F0CAEF2BF007A82A
:106C6000A2EF36F00101800E006F1A0E016F060EC2
:106C7000026F000E036F4BC104F14CC105F14DC111
:106C800006F14EC107F1F5EC39F003BFE8EF36F03D
:106C900050EC38F04BC100F14CC101F14DC102F193
:106CA0004EC103F1078202EC39F018C104F119C199
:106CB00005F11AC106F11BC107F1F80E006FCD0EE8
:106CC000016F660E026F030E036FF5EC39F00E0EC6
:106CD0000C6E00C10BF0F1EC0BF00F0E0C6E01C14D
:106CE0000BF0F1EC0BF0100E0C6E02C10BF0F1EC9E
:106CF0000BF0110E0C6E03C10BF0F1EC0BF00784DE
:106D000001010AEC3BF057C100F158C101F10794B1
:106D10000A0E0C6E00C10BF0F1EC0BF00B0E0C6EBA
:106D200001C10BF0F1EC0BF00C0E0C6E02C10BF07C
:106D3000F1EC0BF00D0E0C6E03C10BF0F1EC0BF04F
:106D4000E8EF36F007AAE8EF36F0078401010AEC15
:106D50003BF057C100F158C101F10794060E0C6ECB
:106D600000C10BF0F1EC0BF0070E0C6E01C10BF043
:106D7000F1EC0BF0080E0C6E02C10BF0F1EC0BF015
:106D8000090E0C6E03C10BF0F1EC0BF0078462C12D
:106D900000F163C101F164C102F165C103F107941F
:106DA000120E0C6E00C10BF0F1EC0BF0130E0C6E1A
:106DB00001C10BF0F1EC0BF0140E0C6E02C10BF0E4
:106DC000F1EC0BF0150E0C6E03C10BF0F1EC0BF0B7
:106DD0000798079A0401805181197F0B0DE09EA846
:106DE000FED714EE00F081517F0BE126E750812B96
:106DF0000F01AD6EEAEF36F005012F51000AD8B44D
:106E00002BEF37F081BA10EF37F015B22BEF37F0D8
:106E100005012F51010AD8B429EF37F022EF37F0DE
:106E200005012F51000AD8B403EF46F005012F5198
:106E3000010AD8B429EF37F000011650050AD8B47A
:106E400003EF46F081B82BEF37F08BEC3DF089EC87
:106E50003EF09CEC45F099EF0EF006013251385DA2
:106E60003351D8A0010F395D800BD8A43CEF37F027
:106E700032C638F633C639F6120006013251365D95
:106E80003351D8A0010F375D800BD8B44CEF37F0E9
:106E900032C636F633C637F6120007841AC632F603
:106EA0001BC633F61CC638F61DC639F62DEC37F076
:106EB0001EC632F61FC633F62DEC37F020C632F66A
:106EC00021C633F62DEC37F01AC632F61BC633F660
:106ED0001CC636F61DC637F63DEC37F01EC632F638
:106EE0001FC633F63DEC37F020C632F621C633F626
:106EF0003DEC37F03851365F3951D8A03929375F2A
:106F00000AEC3BF036C600F137C601F116EC3BF057
:106F100000C13AF601C13BF622C632F623C633F66B
:106F200024C638F625C639F62DEC37F026C632F6DB
:106F300027C633F62DEC37F028C632F629C633F6CD
:106F40002DEC37F022C632F623C633F624C636F6C9
:106F500025C637F63DEC37F026C632F627C633F69F
:106F60003DEC37F028C632F629C633F63DEC37F053
:106F70003851365F3951D8A03929375F0AEC3BF0D8
:106F800036C600F137C601F116EC3BF000C13CF605
:106F900001C13DF62AC632F62BC633F62CC638F6AA
:106FA0002DC639F62DEC37F02EC632F62FC633F645
:106FB0002DEC37F030C632F631C633F62DEC37F013
:106FC0002AC632F62BC633F62CC636F62DC637F651
:106FD0003DEC37F02EC632F62FC633F63DEC37F0D7
:106FE00030C632F631C633F63DEC37F03851365FF5
:106FF0003951D8A03929375F0AEC3BF036C600F189
:1070000037C601F116EC3BF000C13EF601C13FF678
:107010003AC632F63BC633F63CC636F63DC637F6C0
:107020003DEC37F03EC632F63FC633F63DEC37F066
:107030000794120018C100F119C101F11AC102F13F
:107040001BC103F1000E046F000E056F010E066FE9
:10705000000E076F26EC3AF029A145EF38F02051D9
:10706000D8B445EF38F018C100F119C101F11AC1C7
:1070700002F11BC103F1000E046F000E056F0A0E32
:10708000066F000E076F26EC3AF012000101045162
:107090000013055101130651021307510313120087
:1070A0000101186B196B1A6B1B6B12002AC182F459
:1070B0000401300E822770EC0FF02BC182F4040122
:1070C000300E822770EC0FF02CC182F40401300ED8
:1070D000822770EC0FF02DC182F40401300E82275C
:1070E00070EC0FF02EC182F40401300E822770EC98
:1070F0000FF02FC182F40401300E822770EC0FF0E4
:1071000030C182F40401300E822770EC0FF031C1DF
:1071100082F40401300E822770EC0FF032C182F449
:107120000401300E822770EC0FF033C182F40401A9
:10713000300E822770EC0FF012002FC182F4040190
:10714000300E822770EC0FF030C182F40401300E53
:10715000822770EC0FF031C182F40401300E8227D7
:1071600070EC0FF032C182F40401300E822770EC13
:107170000FF033C182F40401300E822770EC0FF05F
:107180001200060E216E060E226E060E236E212EB2
:10719000C7EF38F0222EC7EF38F0232EC7EF38F0B4
:1071A0008B84020E216E020E226E020E236E212EA1
:1071B000D7EF38F0222ED7EF38F0232ED7EF38F064
:1071C0008B941200FF0E226E22C023F0030E216E5C
:1071D0008B84212EE8EF38F0030E216E232EE8EF8A
:1071E00038F08B9422C023F0030E216E212EF6EF8F
:1071F00038F0030E216E233EF6EF38F0222EE4EF36
:1072000038F012000101005305E1015303E102537C
:1072100001E1002BC5EC39F00AEC3BF03951006F6D
:107220003A51016F420E046F4B0E056F000E066F50
:10723000000E076F06EC3AF000C104F101C105F140
:1072400002C106F103C107F118C100F119C101F132
:107250001AC102F11BC103F107B233EF39F0FAECA6
:1072600039F035EF39F0F5EC39F000C118F101C112
:1072700019F102C11AF103C11BF112000AEC3BF033
:1072800059C100F15AC101F1060E08EC0CF0E8CF2B
:1072900004F1070E08EC0CF0E8CF05F1080E08EC3D
:1072A0000CF0E8CF06F1090E08EC0CF0E8CF07F17E
:1072B000F5EC39F000C124F101C125F102C126F13C
:1072C00003C127F1290E046F000E056F000E066F33
:1072D000000E076F06EC3AF0EE0E046F430E056FDA
:1072E000000E066F000E076FFAEC39F024C104F1AE
:1072F00025C105F126C106F127C107F106EC3AF0D8
:1073000000C11CF101C11DF102C11EF103C11FF139
:10731000120E08EC0CF0E8CF04F1130E08EC0CF0A0
:10732000E8CF05F1140E08EC0CF0E8CF06F1150ECD
:1073300008EC0CF0E8CF07F10D0E006F000E016FA6
:10734000000E026F000E036F06EC3AF0180E046F89
:10735000000E056F000E066F000E076F26EC3AF068
:107360001CC104F11DC105F11EC106F11FC107F1C9
:10737000FAEC39F06A0E046F2A0E056F000E066FE4
:10738000000E076FF5EC39F01200BF0EFA6E200EFA
:107390003A6F396BD8900037013702370337D8B0CE
:1073A000D6EF39F03A2FCBEF39F039073A070353CC
:1073B000D8B412000331070B80093F6F03390F0B5C
:1073C000010F396F80EC5FF0406F390580EC5FF0A2
:1073D000405D405F396B3F33D8B0392739333FA91F
:1073E000EBEF39F040513927120001012FEC3BF04F
:1073F000D8B01200010103510719346FF2EC3AF0D2
:10740000D8900751031934AF800F12000101346B7B
:1074100016EC3BF0D8A02CEC3BF0D8B0120001ECFD
:107420003BF00AEC3BF01F0E366F42EC3BF00B35A5
:10743000D8B0F2EC3AF0D8A00335D8B01200362F0D
:1074400015EF3AF034B119EC3BF012000101346B46
:1074500004510511061107110008D8A016EC3BF0E5
:10746000D8A02CEC3BF0D8B01200086B096B0A6B6B
:107470000B6B42EC3BF01F0E366F42EC3BF00751BA
:107480000B5DD8A450EF3AF006510A5DD8A450EF36
:107490003AF00551095DD8A450EF3AF00451085D67
:1074A000D8A063EF3AF00451085F0551D8A0053D1C
:1074B000095F0651D8A0063D0A5F0751D8A0073DD5
:1074C0000B5FD8900081362F3DEF3AF034B119ECC4
:1074D0003BF0346B16EC3BF0D89046EC3BF0075198
:1074E0000B5DD8A480EF3AF006510A5DD8A480EF76
:1074F0003AF00551095DD8A480EF3AF00451085DD7
:10750000D8A08FEF3AF0003F8FEF3AF0013F8FEFB6
:107510003AF0023F8FEF3AF0032BD8B4120034B1A7
:1075200019EC3BF012000101346B16EC3BF0D8B0C3
:1075300012004BEC3BF0200E366F0037013702375C
:10754000033711EE33F00A0E376FE7360A0EE75CA9
:10755000D8B0E76EE552372FA5EF3AF0362F9DEF02
:107560003AF034B12981D89012004BEC3BF0200E58
:10757000366F003701370237033711EE33F00A0E4A
:10758000376FE7360A0EE75CD8B0E76EE552372F63
:10759000C1EF3AF0362FB9EF3AF0D890120001015E
:1075A0000A0E346F200E366F11EE29F03451376F0A
:1075B0000A0ED890E652D8B0E726E732372FDAEF36
:1075C0003AF00333023301330033362FD4EF3AF06D
:1075D000E750FF0FD8A00335D8B0120029B119EC3D
:1075E0003BF01200045100270551D8B0053D01279A
:1075F0000651D8B0063D02270751D8B0073D0327F2
:1076000012000051086F0151096F02510A6F0351B6
:107610000B6F12000101006B016B026B036B120018
:107620000101046B056B066B076B12000335D8A0D4
:1076300012000351800B001F011F021F031F003F98
:1076400029EF3BF0013F29EF3BF0023F29EF3BF0F0
:10765000032B342B032512000735D8A01200075145
:10766000800B041F051F061F071F043F3FEF3BF061
:10767000053F3FEF3BF0063F3FEF3BF0072B342B3E
:10768000072512000037013702370337083709375B
:107690000A370B3712000101296B2A6B2B6B2C6BFD
:1076A0002D6B2E6B2F6B306B316B326B336B12008B
:1076B00001012A510F0B2A6F2B510F0B2B6F2C51ED
:1076C0000F0B2C6F2D510F0B2D6F2E510F0B2E6F9B
:1076D0002F510F0B2F6F30510F0B306F31510F0B9C
:1076E000316F32510F0B326F33510F0B336F12006A
:1076F00000C124F101C125F102C126F103C127F126
:1077000004C100F105C101F106C102F107C103F195
:1077100024C104F125C105F126C106F127C107F1F5
:107720001200899C000EC76E200EC66E9E96C69EE5
:10773000C50EC96EFF0E9EB602D0E82EFCD79E96EF
:10774000C69E000EC96EFF0E9EB602D0E82EFCD774
:10775000C9CF00F69E96C69E000EC96EFF0E9EB65D
:1077600002D0E82EFCD7C9CF01F6898C1200000E9A
:10777000C76E200EC66E899C9E96C69EC80EC96EA8
:10778000FF0E9EB602D0E82EFCD79E96C69E000E37
:10779000C96EFF0E9EB602D0E82EFCD7C9CF02F606
:1077A0009E96C69E000EC96EFF0E9EB602D0E82EB3
:1077B000FCD7C9CF03F69E96C69E000EC96EFF0E7B
:1077C0009EB602D0E82EFCD7C9CF0AF69E96C69E7A
:1077D000000EC96EFF0E9EB602D0E82EFCD7C9CFB0
:1077E0000BF69E96C69E000EC96EFF0E9EB602D088
:1077F000E82EFCD7C9CF12F69E96C69E000EC96E23
:10780000FF0E9EB602D0E82EFCD7C9CF13F6898CA6
:107810001200000EC76E200EC66E899C9E96C69EF4
:10782000E80EC96EFF0E9EB602D0E82EFCD79E96DB
:10783000C69E000EC96EFF0E9EB602D0E82EFCD783
:10784000C9CF1AF69E96C69E000EC96EFF0E9EB652
:1078500002D0E82EFCD7C9CF1BF69E96C69E000E1E
:10786000C96EFF0E9EB602D0E82EFCD7C9CF22F615
:107870009E96C69E000EC96EFF0E9EB602D0E82EE2
:10788000FCD7C9CF23F69E96C69E000EC96EFF0E8A
:107890009EB602D0E82EFCD7C9CF2AF69E96C69E89
:1078A000000EC96EFF0E9EB602D0E82EFCD7C9CFDF
:1078B0002BF6898C1200000EC76E200EC66E899CB6
:1078C0009E96C69E240EC96EFF0E9EB602D0E82E6E
:1078D000FCD79E96C69EE40EC96EFF0E9EB602D0E1
:1078E000E82EFCD7898C899C9E96C69E200EC96E78
:1078F000FF0E9EB602D0E82EFCD79E96C69E5F0E67
:10790000C96EFF0E9EB602D0E82EFCD7898C899CEA
:107910009E96C69E210EC96EFF0E9EB602D0E82E20
:10792000FCD79E96C69EC00EC96EFF0E9EB602D0B4
:10793000E82EFCD7898C899C9E96C69E260EC96E21
:10794000FF0E9EB602D0E82EFCD79E96C69E000E75
:10795000C96EFF0E9EB602D0E82EFCD7898C1200AD
:10796000000EC76E200EC66E899C9E96C69E200E87
:10797000C96EFF0E9EB602D0E82EFCD79E96C69E1C
:10798000000EC96EFF0E9EB602D0E82EFCD7898C81
:10799000120010A806D08994000EC76E220EC66E83
:1079A00005D08984000EC76E220EC66E050EE82E25
:1079B000FED7120010A802D0898401D08994050E48
:1079C000E82EFED71200C9EC3CF09E96C69E000E33
:1079D000C96EFF0E9EB602D0E82EFCD79E96C69EBC
:1079E000000EC96EFF0E9EB602D0E82EFCD7C9CF9E
:1079F000AFF59E96C69E000EC96EFF0E9EB602D0D3
:107A0000E82EFCD7C9CFB0F59E96C69E000EC96E73
:107A1000FF0E9EB602D0E82EFCD7C9CFB1F59E96D8
:107A2000C69E000EC96EFF0E9EB602D0E82EFCD791
:107A3000C9CFB2F59E96C69E000EC96EFF0E9EB6C9
:107A400002D0E82EFCD7C9CFB3F59E96C69E000E95
:107A5000C96EFF0E9EB602D0E82EFCD7C9CFB4F592
:107A60009E96C69E000EC96EFF0E9EB602D0E82EF0
:107A7000FCD7C9CFB5F5DAEC3CF01200C9EC3CF00C
:107A80009E96C69E800EC96EFF0E9EB602D0E82E50
:107A9000FCD79E96C69EAFC5C9FFFF0E9EB602D00C
:107AA000E82EFCD79E96C69EB0C5C9FFFF0E9EB6B7
:107AB00002D0E82EFCD79E96C69EB1C5C9FFFF0E28
:107AC0009EB602D0E82EFCD79E96C69EB2C5C9FFD0
:107AD000FF0E9EB602D0E82EFCD79E96C69EB3C57A
:107AE000C9FFFF0E9EB602D0E82EFCD79E96C69E1A
:107AF000B4C5C9FFFF0E9EB602D0E82EFCD79E96F5
:107B0000C69EB5C5C9FFFF0E9EB602D0E82EFCD7B3
:107B1000DAEC3CF01200C9EC3CF09E96C69E070ED3
:107B2000C96EFF0E9EB602D0E82EFCD79E96C69E6A
:107B3000000EC96EFF0E9EB602D0E82EFCD7C9CF4C
:107B4000AFF59E96C69E000EC96EFF0E9EB602D081
:107B5000E82EFCD7C9CFB0F59E96C69E000EC96E22
:107B6000FF0E9EB602D0E82EFCD7C9CFB1F59E9687
:107B7000C69E000EC96EFF0E9EB602D0E82EFCD740
:107B8000C9CFB2F5DAEC3CF0C9EC3CF09E96C69E4B
:107B900025C0C9FFFF0E9EB602D0E82EFCD79E96E8
:107BA000C69E000EC96EFF0E9EB602D0E82EFCD710
:107BB000C9CFB6F5DAEC3CF01200C9EC3CF09E9669
:107BC000C69E870EC96EFF0E9EB602D0E82EFCD769
:107BD0009E96C69EAFC5C9FFFF0E9EB602D0E82E88
:107BE000FCD79E96C69EB0C5C9FFFF0E9EB602D0BA
:107BF000E82EFCD79E96C69EB1C5C9FFFF0E9EB665
:107C000002D0E82EFCD79E96C69EB2C5C9FFFF0ED5
:107C10009EB602D0E82EFCD7DAEC3CF0C9EC3CF082
:107C20009E96C69E26C0C9FFFF0E9EB602D0E82EC5
:107C3000FCD79E96C69EB6C5C9FFFF0E9EB602D063
:107C4000E82EFCD7DAEC3CF01200C9EC3CF09E9632
:107C5000C69E870EC96EFF0E9EB602D0E82EFCD7D8
:107C60009E96C69E000EC96EFF0E9EB602D0E82EEE
:107C7000FCD79E96C69E800EC96EFF0E9EB602D0A1
:107C8000E82EFCD79E96C69E800EC96EFF0E9EB64D
:107C900002D0E82EFCD79E96C69E800EC96EFF0EBF
:107CA0009EB602D0E82EFCD7DAEC3CF01200C9EC0C
:107CB0003CF09E96C69E870EC96EFF0E9EB602D001
:107CC000E82EFCD79E96C69E000EC96EFF0E9EB68D
:107CD00002D0E82EFCD79E96C69E000EC96EFF0EFF
:107CE0009EB602D0E82EFCD79E96C69E800EC96E28
:107CF000FF0E9EB602D0E82EFCD79E96C69E800E42
:107D0000C96EFF0E9EB602D0E82EFCD7DAEC3CF02E
:107D1000120010A817D0C9EC3CF09E96C69E8F0E9C
:107D2000C96EFF0E9EB602D0E82EFCD79E96C69E68
:107D3000000EC96EFF0E9EB602D0E82EFCD7DAEC1C
:107D40003CF012008BEC3DF0120010A82DD0C9ECD5
:107D50003CF09E96C69E26C0C9FFFF0E9EB602D07E
:107D6000E82EFCD79E96C69E450EC96EFF0E9EB6A7
:107D700002D0E82EFCD7DAEC3CF0C9EC3CF09E9641
:107D8000C69E8F0EC96EFF0E9EB602D0E82EFCD79F
:107D90009E96C69E000EC96EFF0E9EB602D0E82EBD
:107DA000FCD7DAEC3CF01200C9EC3CF09E96C69E83
:107DB00026C0C9FFFF0E9EB602D0E82EFCD79E96C5
:107DC000C69E010EC96EFF0E9EB602D0E82EFCD7ED
:107DD000DAEC3CF0C9EC3CF09E96C69E910EC96E62
:107DE000FF0E9EB602D0E82EFCD79E96C69EA50E2C
:107DF000C96EFF0E9EB602D0E82EFCD7DAEC3CF03E
:107E00001200C9EC3CF09E96C69E26C0C9FFFF0E2C
:107E10009EB602D0E82EFCD79E96C69E810EC96EF5
:107E2000FF0E9EB602D0E82EFCD7DAEC3CF0120032
:107E3000C9EC3CF09E96C69E26C0C9FFFF0E9EB6BA
:107E400002D0E82EFCD79E96C69E010EC96EFF0E8C
:107E50009EB602D0E82EFCD7DAEC3CF01200C9EC5A
:107E60003CF09E96C69E910EC96EFF0E9EB602D045
:107E7000E82EFCD79E96C69EA50EC96EFF0E9EB636
:107E800002D0E82EFCD7DAEC3CF01200C9EC3CF052
:107E90009E96C69E910EC96EFF0E9EB602D0E82E2B
:107EA000FCD79E96C69E000EC96EFF0E9EB602D0EF
:107EB000E82EFCD7DAEC3CF012000501256B266BAE
:107EC000276B286B899A400EC76E200EC66E9E9651
:107ED000C69E030EC96EFF0E9EB602D0E82EFCD7DA
:107EE0009E96C69E27C5C9FFFF0E9EB602D0E82EFD
:107EF000FCD79E96C69E26C5C9FFFF0E9EB602D031
:107F0000E82EFCD79E96C69E25C5C9FFFF0E9EB6DD
:107F100002D0E82EFCD79E96C69EC952FF0E9EB692
:107F200002D0E82EFCD7898A0F01C950FF0A01E16F
:107F3000120005012E51130A05E005012E51170A02
:107F40000CE012000501E00E256FFF0E266F0F0EEC
:107F5000276F000E286FB6EF3FF00501E00E256F8A
:107F6000FF0E266FFF0E276F000E286F899A400EB6
:107F7000C76E200EC66E9E96C69E030EC96EFF0E7D
:107F80009EB602D0E82EFCD79E96C69E27C5C9FF96
:107F9000FF0E9EB602D0E82EFCD79E96C69E26C542
:107FA000C9FFFF0E9EB602D0E82EFCD79E96C69E55
:107FB00025C5C9FFFF0E9EB602D0E82EFCD79E96BF
:107FC000C69EC952FF0E9EB602D0E82EFCD7898A03
:107FD0000F01C950FF0A1DE005012E51130A05E0EB
:107FE00005012E51170A0BE012000501000E256F46
:107FF000000E266F100E276F000E286F120005016D
:10800000000E256F000E266F000E276F010E286FE1
:1080100012000501256B266B276B286B05012E517D
:10802000130A05E005012E51170A0CE012000501A4
:10803000000E216F000E226F080E236F000E246FBA
:108040002BEF40F00501000E216F000E226F800E15
:10805000236F000E246F21C500F122C501F123C555
:1080600002F124C503F125C504F126C505F127C594
:1080700006F128C507F146EC38F000C125F501C12D
:1080800026F502C127F503C128F5899A400EC76E6F
:10809000200EC66E9E96C69E030EC96EFF0E9EB63D
:1080A00002D0E82EFCD79E96C69E27C5C9FFFF0EBC
:1080B0009EB602D0E82EFCD79E96C69E26C5C9FF66
:1080C000FF0E9EB602D0E82EFCD79E96C69E25C512
:1080D000C9FFFF0E9EB602D0E82EFCD79E96C69E24
:1080E000C952FF0E9EB602D0E82EFCD7898AC9502D
:1080F000FF0A08E104C125F505C126F506C127F5EB
:1081000007C128F5D89005012433233322332133C6
:108110002151E00B216F0501216796EF40F02267A6
:1081200096EF40F0236796EF40F024672BEF40F086
:108130000501200E2527E86A2623E86A2723E86A36
:1081400028231200E86A05012E51130A06E00501F2
:108150002E51170A0BE0020E120005012851000AE9
:1081600003E12751F00B07E0010E12000501285131
:10817000000A01E0010E120029C500F12AC501F133
:108180002BC502F12CC503F125C504F126C505F167
:1081900027C506F128C507F1F5EC39F003BF120039
:1081A000A2EC40F0D8A434EF41F0899A400EC76E9B
:1081B000200EC66E9E96C69E060EC96EFF0E9EB619
:1081C00002D0E82EFCD7898A899A9E96C69E020E16
:1081D000C96EFF0E9EB602D0E82EFCD79E96C69EB4
:1081E00027C5C9FFFF0E9EB602D0E82EFCD79E968B
:1081F000C69E26C5C9FFFF0E9EB602D0E82EFCD74C
:108200009E96C69E25C5C9FFFF0E9EB602D0E82EDB
:10821000FCD79E96C69E000EC96EFF0E9EB602D07B
:10822000E82EFCD7898A899A9E96C69E050EC96E4D
:10823000FF0E9EB602D0E82EFCD79E96C69EC9526F
:10824000FF0E9EB602D0E82EFCD7C9B01DEF41F05C
:10825000898A0501200E2527E86A2623E86A272354
:10826000E86A2823BCEF40F01200899A400EC76EDE
:10827000200EC66E9E96C69E060EC96EFF0E9EB658
:1082800002D0E82EFCD7898A899A9E96C69EC70E90
:10829000C96EFF0E9EB602D0E82EFCD7898A050172
:1082A000256B266B276B286B1200899A400EC76ED0
:1082B000200EC66E9E96C69E050EC96EFF0E9EB619
:1082C00002D0E82EFCD79E96C69EC952FF0E9EB6DF
:1082D00002D0E82EFCD7C9CF37F5898A1200899AD7
:1082E000400EC76E200EC66E9E96C69EB90EC96E13
:1082F000FF0E9EB602D0E82EFCD7898A1200899A1A
:10830000400EC76E200EC66E9E96C69EAB0EC96E00
:10831000FF0E9EB602D0E82EFCD7898AFF0EE82E0B
:10832000FED71200A2EC40F0D8A41200899A400EA9
:10833000C76E200EC66E9E96C69E030EC96EFF0EB9
:108340009EB602D0E82EFCD79E96C69E27C5C9FFD2
:10835000FF0E9EB602D0E82EFCD79E96C69E26C57E
:10836000C9FFFF0E9EB602D0E82EFCD79E96C69E91
:1083700025C5C9FFFF0E9EB602D0E82EFCD79E96FB
:10838000C69EC952FF0E9EB602D0E82EFCD7898A3F
:108390000F01C950FF0AD8A40DEF45F00501FE0EEC
:1083A000376F0501FF0E536FFF0E546FFF0E556FB1
:1083B000FF0E566F15A637991586E3EC3CF0AFC556
:1083C00038F5B0C539F5B1C53AF5B2C53BF5B3C519
:1083D0003CF5B4C53DF5B5C53EF50784BAC166F1B7
:1083E000BBC167F1BCC168F1BDC169F14BC14FF1BF
:1083F0004CC150F14DC151F14EC152F157C159F12B
:1084000058C15AF100011650010AD8B416EF42F0D3
:1084100000011650020AD8B43BEF42F0000116509A
:10842000040AD8B460EF42F00DEF45F00501476B48
:10843000486B496B4A6B05014B6B4C6B4D6B4E6B3C
:1084400005014F6B506B516B526B8BA0379BF4EC5B
:108450002BF000C1DAF101C1DBF102C1DCF103C193
:10846000DDF100C13FF501C140F502C141F503C195
:1084700042F57FEF42F00501476B486B496B4A6B51
:1084800005014B6B4C6B4D6B4E6B05014F6B506B8D
:10849000516B526BF4EC2BF000C1DAF101C1DBF14E
:1084A00002C1DCF103C1DDF1F1EC2CF000C147F5B4
:1084B00001C148F502C149F503C14AF50DEF45F088
:1084C000379BDAC13FF5DBC140F5DCC141F5DDC1C9
:1084D00042F5F4EC2BF000C14BF501C14CF502C1A3
:1084E0004DF503C14EF5F1EC2CF000C14FF501C183
:1084F00050F502C151F503C152F57FEF42F005017D
:1085000061678AEF42F062678AEF42F063678AEF41
:1085100042F064678EEF42F0A3EF42F0DAC100F15F
:10852000DBC101F1DCC102F1DDC103F161C504F180
:1085300062C505F163C506F164C507F1F5EC39F0D4
:1085400003BF0DEF45F059C143F55AC144F5B9C514
:1085500045F54DEC37F036C649F537C64AF5060104
:108560004067BAEF42F04167BAEF42F04267BAEFB4
:1085700042F04367BEEF42F0CFEF42F00AEC3BF02F
:1085800010EC3BF036C600F137C601F140C604F1ED
:1085900041C605F1F5EC39F003AF0DEF45F00101EF
:1085A000036B026B1AC600F11BC601F101AFDDEFD0
:1085B00042F0FF0E026FFF0E036F0101076B066BA7
:1085C0001CC604F11DC605F105AFEBEF42F0FF0E2E
:1085D000066FFF0E076FFAEC39F00101076B066BAF
:1085E0001EC604F11FC605F105AFFBEF42F0FF0EFA
:1085F000066FFF0E076FFAEC39F00101076B066B8F
:1086000020C604F121C605F105AF0BEF43F0FF0EC4
:10861000066FFF0E076FFAEC39F0D89001010333B3
:10862000023301330033D8900101033302330133A5
:10863000003300C14BF501C14CF50101036B026B26
:1086400022C600F123C601F101AF2BEF43F0FF0E6C
:10865000026FFF0E036F0101076B066B24C604F166
:1086600025C605F105AF39EF43F0FF0E066FFF0E8B
:10867000076FFAEC39F00101076B066B26C604F1AF
:1086800027C605F105AF49EF43F0FF0E066FFF0E59
:10869000076FFAEC39F00101076B066B28C604F18D
:1086A00029C605F105AF59EF43F0FF0E066FFF0E27
:1086B000076FFAEC39F0D89001010333023301332C
:1086C0000033D8900101033302330133003300C17A
:1086D0004DF501C14EF50101036B026B2AC600F195
:1086E0002BC601F101AF79EF43F0FF0E026FFF0ED1
:1086F000036F0101076B066B2CC604F12DC605F153
:1087000005AF87EF43F0FF0E066FFF0E076FFAEC21
:1087100039F00101076B066B2EC604F12FC605F177
:1087200005AF97EF43F0FF0E066FFF0E076FFAECF1
:1087300039F00101076B066B30C604F131C605F153
:1087400005AFA7EF43F0FF0E066FFF0E076FFAECC1
:1087500039F0D89001010333023301330033D8904C
:108760000101033302330133003300C14FF501C16E
:1087700050F50101036B026B02C600F103C601F163
:1087800001AFC7EF43F0FF0E026FFF0E036F010151
:10879000076B066B04C604F105C605F105AFD5EFFE
:1087A00043F0FF0E066FFF0E076FFAEC39F0010180
:1087B000076B066B06C604F107C605F105AFE5EFCA
:1087C00043F0FF0E066FFF0E076FFAEC39F0010160
:1087D000076B066B08C604F109C605F105AFF5EF96
:1087E00043F0FF0E066FFF0E076FFAEC39F0D890DA
:1087F00001010333023301330033D8900101033305
:1088000002330133003300C151F501C152F50101BA
:10881000036B026B0AC600F10BC601F101AF15EF45
:1088200044F0FF0E026FFF0E036F0101076B066B32
:108830000CC604F10DC605F105AF23EF44F0FF0EA1
:10884000066FFF0E076FFAEC39F00101076B066B3C
:108850000EC604F10FC605F105AF33EF44F0FF0E6D
:10886000066FFF0E076FFAEC39F00101076B066B1C
:1088700010C604F111C605F105AF43EF44F0FF0E39
:10888000066FFF0E076FFAEC39F0D8900101033341
:10889000023301330033D890010103330233013333
:1088A000003300C153F501C154F50101036B026BA4
:1088B00012C600F113C601F101AF63EF44F0FF0EE1
:1088C000026FFF0E036F0101076B066B14C604F104
:1088D00015C605F105AF71EF44F0FF0E066FFF0EF0
:1088E000076FFAEC39F00101076B066B16C604F14D
:1088F00017C605F105AF81EF44F0FF0E066FFF0EBE
:10890000076FFAEC39F00101076B066B18C604F12A
:1089100019C605F105AF91EF44F0FF0E066FFF0E8B
:10892000076FFAEC39F0D8900101033302330133B9
:108930000033D8900101033302330133003300C107
:1089400055F501C156F50501210E326F899A400E89
:10895000C76E200EC66E9E96C69E060EC96EFF0E90
:108960009EB602D0E82EFCD7898A899A9E96C69E2A
:10897000020EC96EFF0E9EB602D0E82EFCD79E9660
:10898000C69E27C5C9FFFF0E9EB602D0E82EFCD7B3
:108990009E96C69E26C5C9FFFF0E9EB602D0E82E43
:1089A000FCD79E96C69E25C5C9FFFF0E9EB602D077
:1089B000E82EFCD725EE37F0322F02D0EBEF44F053
:1089C0009E96C69EDECFC9FFFF0E9EB602D0E82E51
:1089D000FCD7DCEF44F0898A899A9E96C69E050EE4
:1089E000C96EFF0E9EB602D0E82EFCD79E96C69E9C
:1089F000C952FF0E9EB602D0E82EFCD7C9B0F6EFE2
:108A000044F0898A0501200E2527E86A2623E86AB2
:108A10002723E86A2823C1EC38F015900794120048
:108A200021C500F122C501F123C502F124C503F1DE
:108A3000899A400EC76E200EC66E9E96C69E0B0E7D
:108A4000C96EFF0E9EB602D0E82EFCD79E96C69E3B
:108A500002C1C9FFFF0E9EB602D0E82EFCD79E963B
:108A6000C69E01C1C9FFFF0E9EB602D0E82EFCD7FC
:108A70009E96C69E00C1C9FFFF0E9EB602D0E82E8C
:108A8000FCD79E96C69EC952FF0E9EB602D0E82E17
:108A9000FCD725EE37F00501200E326F9E96C69E5C
:108AA000C952FF0E9EB602D0E82EFCD7C9CFDEFF1A
:108AB000322F4EEF45F0898A1200899A400EC76E18
:108AC000200EC66E9E96C69E900EC96EFF0E9EB676
:108AD00002D0E82EFCD79E96C69E000EC96EFF0EF1
:108AE0009EB602D0E82EFCD79E96C69E000EC96E9A
:108AF000FF0E9EB602D0E82EFCD79E96C69E000EB4
:108B0000C96EFF0E9EB602D0E82EFCD79E96C69E7A
:108B1000C952FF0E9EB602D0E82EFCD7C9CF2DF564
:108B20009E96C69EC952FF0E9EB602D0E82EFCD776
:108B3000C9CF2EF5898A1200E3EC3CF005012F51D4
:108B4000010A5FE005012F51020A16E005012F51CD
:108B5000030A19E005012F51040A24E005012F51F1
:108B6000050A2BE005012F51060A39E005012F51B6
:108B7000070A3FE001EF46F0602FFFEF45F05FC5C9
:108B800060F501EF46F0B0C500F101010F0E0017CE
:108B900001010051000A35E001010051050A31E0F0
:108BA000FFEF45F0B0C500F101010F0E0017010104
:108BB0000051000A26E0FFEF45F00501B051000A20
:108BC00020E00501B051150A1CE00501B051300A42
:108BD00018E00501B051450A14E0FFEF45F005012A
:108BE000B051000A0EE00501B051300A0AE0FFEF73
:108BF00045F00501B051000A04E0FFEF45F0159083
:108C00001200158012008B90C1EC38F0B9C5E8FF56
:108C1000D70802E3C1EC38F0B9C5E8FFC80802E3A1
:108C2000C1EC38F0B9C5E8FFB90802E3C1EC38F08F
:108C3000B9C5E8FFAA0802E3C1EC38F0B9C5E8FFFE
:108C40009B0802E3C1EC38F06FEC41F0F29CF29E1D
:108C50008B94C69AC290B0EC3CF09482948C720EC5
:108C6000D36ED3A4FED789968A909390F29AF29409
:108C70009D909E909D929E92F298F29289EC3EF089
:108C8000FF0EE8CF00F0E82EFED7002EFCD7F290C2
:108C9000F286815081A84FEF46F0F29E0300700EDD
:108CA000D36EF296F29015840380E2EC38F03EEF3A
:028CB0000CF0C6
:10BF0000E844F926000C160C2B0C3F0C520C640C68
:10BF1000760C860C960CA50CB30CC10CCF0CDC0C6B
:06BF2000E80CF40C000C1B
:0200000400F00A
:0100C800FE39
:00000001FF
